:020000041100E9
:10300000002373B52B4D2C4C28006361022601F080
:103010006DF94021FE2221742800284B009601F012
:10302000B7F9002836D1217CFF222800244B0096D6
:1030300001F0AEF900282DD1224BA2899A4226D167
:10304000E389214A93420DD1204B6361204B2268D2
:10305000002A03D1002B01D043CB43C4280001F048
:1030600083F973BD1B4A934201D00023EFE71A4B4B
:103070001A4A1B68934206D9C02304222800217CE7
:103080009B0001F0FBF9114B6361154BDFE7002357
:103090002374EAE7CC233821AC2228009B01217459
:1030A00001F0ECF90028F2D10E4B63610E4BE38185
:1030B0000E4BCCE7743CFF1F1C5CFF1F285CFF1FFE
:1030C0002A5CFF1F595900008305000019410011B7
:1030D000D8BC001182150000405CFF1F8713000060
:1030E000E4BC0011D1410011AAAAFFFFCCBC001121
:1030F000F7B5164B0192C318021D002000938823D8
:103100005B05D3181B685C1C1AD09CB2402C18D8E5
:103110008D781E0CAC466746CD782D023D43AE42FD
:1031200006D1019800280ED110000C70240A4C70B2
:1031300003249BB20733A343D218009B9A42DED3E9
:10314000FEBD4432F9E71000FAE7C046FC0F00006C
:10315000802213B503000324019189B25201073183
:103160009B18A14304305A1A88235B05C3181B68B7
:10317000591C03D190429241104016BD99B240298A
:1031800007D80B000733A343C0189042ECD30020AC
:10319000F3E74430F9E7134B134A1B68126810B584
:1031A000FA24934201D81A00F824104BE4021B6859
:1031B0009A4210D813000E4A12689A420ED3013375
:1031C00007D1F823DB029C4203D10A49054808F0E5
:1031D0004FFA200010BDFC24E402ECE7FE24E402D8
:1031E000F7E7C04600C0071100D0071100E0071143
:1031F00000F00711FFFFFF7FF0B59BB015000490B2
:103200000391402A00D9A0E006AB59801A80FFF74D
:10321000C2FF0400042816D9002206A9FFF768FFA0
:10322000052810D906AB1B88AB420CD1002D07D066
:10323000514B2A000499C01808F042FC002802D122
:1032400001201BB0F0BD06AB1D8020000699FFF7E2
:103250007FFF041E7BD1069B0793FFF79CFF802313
:103260005B01C618802307001B039E4201D3F8268A
:10327000F60288235B05F31801931B68013302D023
:10328000019808F005FA3D49019808F0F1F93B1D55
:103290000293331D05938822029B52059B181B68DD
:1032A00008935A1C3CD044219AB20091402A04D879
:1032B0000320D11D814389B2009103991B0C8B42DD
:1032C00024D0402A22D80122300008A9FFF710FF9D
:1032D000021E1BD1380008A9FFF70AFF04000428CA
:1032E00031D9009A059B9B1880225201B218934253
:1032F00040D288235B05C118009A09A808F0F0FAAB
:103300001D4B009A09A9F01808F042FA009A029B96
:103310009446634402931A4B029AFB189A42BAD31A
:1033200088235B05FC1821680198013908F0A0F991
:10333000200008F0ADF9039A07AB5A8030000799D6
:10334000FFF706FF0400002C03D1002079E70428D2
:10335000FBD988235B05E018069908F089F9032357
:10336000EA1C9A4300D16BE7034B0499E01808F07C
:103370000FFA65E70424ECE704000011FFFFFF7F6C
:10338000F80F0000F7B505001400402A21D80027E7
:1033900001AE71803780FFF7FEFE042816D93A008F
:1033A0003100FFF7A5FE042810D93688BC420BD0A7
:1033B000BD4209D0221CB44200D9321C064B92B245
:1033C000C118280008F08CFA30B2FEBDC04300B22C
:1033D000FBE703204042F8E70400001137B5042260
:1033E00004000D0001A81649FFF7CCFF02000428D5
:1033F0000BD1019BA34208D3AB4204D0104901A8D2
:103400000195FFF7F9FE01203EBD0E4C2368200018
:10341000019308F03DF9019920000139019108F06C
:1034200027F980235B01E418074B9C42EED104226C
:10343000034901A80195FFF7DFFE0020E4E7C0463D
:103440005555000000C007110000081130B589B0C3
:1034500008F0DEF810226946254808F0B9F9254B36
:10346000009A9A420ED1019B029A0F2B33D8002169
:1034700001240698013B08D2002900D00292029B49
:10348000013331D10023029325E0551CF2D1020013
:103490002100EFE710341022200004A908F098F969
:1034A000029B013301D1069B0293882304995B059B
:1034B000C918059B06981A03120B049105928142C4
:1034C00003D02B4201D108F00BFA019B013B019381
:1034D000019B002BDED1029B002B03D004930498A8
:1034E0004168084709B030BDE025014C2D03EFE7E6
:1034F00000000111504859368022F8B5964C974B80
:10350000D200002120001C6008F012FA2300944A27
:1035100088331A60934B1A786A23002A00D011333B
:10352000E3620A232365904B37221B780821A363AB
:103530008E4B6018E361102323628D4B3B25636142
:10354000C823DB00A36123008C331A602823013ACF
:10355000E26321646364C267043A201DC2672000ED
:10356000BC3005602000C03001602000C430036022
:1035700020000635CC3005602000083DC8300560CD
:103580002000D03002602200D43211602200D832F4
:10359000136022000226E032200016604222DC3056
:1035A000026020001B3DE43005602000E83001602F
:1035B0002000EC30036023000520F4331860230062
:1035C000F0331A602300183290331A6023009433CA
:1035D000196023001E3A98331A60AF23DB00236082
:1035E000644BFA252363644B6448A3642300B93217
:1035F000FC33FF32AD00A260E56022611D60A06275
:103600007320E0656D386065A065FA2796203F015C
:103610008000E76465625960A0660920E0660020CA
:10362000616757496666E167564E57492667A06746
:103630000F601527676027001A219C373960270023
:103640000731A037396027004B49A837396021007E
:10365000F8310D6021006427A4310F6021005F3F25
:10366000AC310F602100033FB0310F602700B43749
:103670003D00C8272F6027003825B83738609D6087
:10368000424D96215D64424D8900DD61414D1962D4
:103690005D62F53DFF3D9D621E253949DD66596637
:1036A000996499673C49DE651E6618675867D96753
:1036B000BE233A495B00E1508130394BFF30235043
:1036C00004302150C42149006350C623E4205B002C
:1036D000E2500433E2503349334A344BD160344929
:1036E000800019503349E938FF3819503249043005
:1036F000195032493248D16132491163324951631C
:103700001900F4310860CE20304940001160304982
:10371000195019002F48F83108602F49D1658221CE
:103720002E4A89005A501A002D490832D1671A00D2
:103730002C49B432116088212B4A89005A501A0052
:103740002A49883211602A4ADA6408F089F901208E
:1037500008F06EF9F8BDC0460004FF1FC85EFF1FE9
:10376000A069FF1FB03EFF1F4A0AFF1F3A07000073
:1037700080C3C9019A02000050C300006A1800000B
:1037800088130000204E0000F009FF1F6509FF1F8D
:1037900068100000C4090000DC05000040420F0072
:1037A00010270000D91AFF1FFC00FF1F0000FF1F99
:1037B0009527FF1FD92AFF1F7129FF1F251EFF1FF5
:1037C0007523FF1F411EFF1FED1FFF1FB11DFF1FB0
:1037D0000124FF1FE924FF1FD918FF1FB923FF1F72
:1037E000C921FF1FD521FF1FB11CFF1F691DFF1F2E
:1037F0009D1CFF1FF0B5022501245E4B91B01D708A
:1038000002935D4B5D4E1C705D4F03933368002146
:103810002800BB7006F0EEFD280006F0E5FC002352
:10382000984205D0BA78552A02D0332A00D095E0C4
:10383000336007F0B5FEFFF75FFE1F220124002171
:10384000504B36251A70504B1C70504B1970504B12
:1038500019689143163A0A431A6060221968914325
:10386000403A0A431A6007F073FF07F051FFC12086
:10387000FF21484B80001A588A431A50C5229200F3
:1038800098588843BF390143995098584249084095
:103890008021C9010143802099509958C00509022F
:1038A000090A0143995080213C48490108F000F978
:1038B0000323220000933A4901943A4808F078F82B
:1038C0002E22394904A808F00BF802AB04ACED181D
:1038D00061782078023406F0A7FCA542F8D1334C79
:1038E000334B226803201A40A023DB0213432360DA
:1038F000802322689B041343236022682D4B1A40C7
:1039000080239B03134323602B4A2C4B934200D804
:10391000012008F05DF907F073FF80232268DB04C3
:1039200013432360029B187808F04AF8039B187829
:10393000C0B207F0A5FE07F0B3FF2149042008F04C
:1039400097F806F08BFE00F0ABF800F0EDFD00F00C
:103950007FFE00F00FFA002011B0F0BD00932100AF
:10396000174A042008F044F88023DB059C62FFF727
:103970006DFD5EE74A0AFF1FB03EFF1F34F00040B6
:103980004C5CFF1F480AFF1F490AFF1F680AFF1F00
:10399000BCF0004000E100E0FF00FFFFB43EFF1F6D
:1039A0003851FF1FB44EFF1FF0BB001114F0004050
:1039B000FF7FF8FFFFFF9FFF0080FF1FA069FF1F31
:1039C0003B00010870B500252549264A26484D636D
:1039D00008CA1B051B0DED188242F9D10026802272
:1039E000224B92058B630921214B224C1E62224BF4
:1039F0001120DA67214BDA688A43DA609A68204935
:103A00000A409A60266008F06BF8112008F0A0F8D0
:103A1000636C1C4A134063641B4C1C4A6C43200CAF
:103A20000400642390420AD8FA223300D200904264
:103A300005D9174B0A21C01807F06AFFC3B2154A0F
:103A400011201372D48008F06BF8134B1B78002BF5
:103A500004D1124B1021187807F052FF70BDC046F8
:103A6000000005408807054000080540FF010000F0
:103A700000F000400038004004E100E03CF000406D
:103A8000FFDFFFFFFFFDFFFFAE060000B70B0000EA
:103A900030F8FFFF345CFF1F6E5EFF1F6C5CFF1F82
:103AA000002210B51100112007F01AFE10BD000011
:103AB000F8B500230925374F374C3B62E3681120E6
:103AC000AB43E36008F044F8112008F009F8112036
:103AD00007F0AEFE40232268802613432360802334
:103AE0006268DB0213436360A3682C4A3343A3601C
:103AF000A36828001340A3608023A2689B0113439E
:103B00001022A360236C022193432364236C0F3A99
:103B10001343236480235B013B62226B204B1A40DA
:103B20002263626B1A406263A26B1A40A263E26B6B
:103B30001340E363E3681B4A1340E36006F074FB41
:103B40002800012106F084FC8023174A9B00516C59
:103B500011200B43536408F043F8FD21134B144A22
:103B600089005A508023C720E26B5B031343E36351
:103B7000E36880001D430F4BE56019580E4A114061
:103B8000802212020A431A50802292051A600B4BBF
:103B90005E63F8BD00F000403CF00040FFFFDFFF37
:103BA000EFFFEFFFFFFF7FFF003800400000FF1F27
:103BB000C539001100E100E0FF00FFFF00000540F3
:103BC00030B503A804880B20002C0ED14968074D9E
:103BD00008784978090201430A20A94205D1012148
:103BE00020001980024B1B7A137030BD192A000087
:103BF000345CFF1FF7B5150008AA16884A680F4FF6
:103C000014785278120222430A24BA4214D10122B3
:103C1000DBB2019200962A0007F05AFC041E0BD179
:103C2000074B1B68002B07D068782A7800021043E6
:103C300042425041013098472000FEBD0229000059
:103C4000B85BFF1F30B5012503790400BFB02B42DC
:103C500011D00A49408806F0A7FF28420BD0084B34
:103C600001A95B8D4D800B80064B00221B7A60887A
:103C70000B7104F0A1F83FB030BDC046B05BFF1F30
:103C8000E83AFF1F345CFF1F10B50549054806F0F0
:103C900041FF0421044A054806F0FEFE10BDC0465F
:103CA000B05BFF1FFFFF000020BC0011E83AFF1FC0
:103CB00010B5024804F002FF10BDC046453C00119B
:103CC000062310B5837010330371443B43712A33CC
:103CD00083714433C37100230222012103720E4B0E
:103CE000027041701C8881724472197A0273C17229
:103CF0009A784273DA7882730322C2731A79027453
:103D00005A7942740C2282749A79C274DB790375F1
:103D10001123C370152010BD345CFF1F10B5142093
:103D200007F03EFF124B14220021186007F000FE3E
:103D3000002007F005FD012007F062FE022007F0D9
:103D40000FFF032004F05EF9042006F073F905204C
:103D500003F09CFB062004F069F8072001F032FA1A
:103D6000082006F079FE092001F01AF810BDC046BF
:103D7000BC5BFF1F07F0DCFC012007F049FE07F0E9
:103D80001FFD0000094B10B50400984205D0012921
:103D900004D12000064906F0BDFE10BD0229FCD169
:103DA000013904F049FE0028F3D0F6E7FEFF0000D9
:103DB000E25BFF1F70B50D7A100004AA2C00168874
:103DC00010221440154220D1002E20D10A78022A58
:103DD00018D14A68517815780E4A09022943914250
:103DE00005D00D4A914209D01C800A2404E0142217
:103DF0000A491A8007F074FD200070BD0C220849A2
:103E00001A80F7E71C800124F6E70824F4E70B2466
:103E1000F2E7C046F3FF0000F4FF0000403DFF1F43
:103E2000FCBC001110B504000749084806F072FEFA
:103E3000074804F083FD0020E40704D50721054A64
:103E4000054806F029FE10BDE25BFF1FFFFF0000E2
:103E5000853D001164BC00112C3BFF1F00B50C4BCD
:103E6000BFB01A780B4902A800F0ACFC6B4680B2D8
:103E7000D880002809D06A46074B01A91B88938087
:103E8000064B0022188803F097FF3FB000BDC046E4
:103E9000C05BFF1FC15BFF1F863BFF1F903CFF1FE6
:103EA00000B50C4BBFB01A780B4902A801F0CAFE4E
:103EB0006B4680B2D880002809D06A46074B01A91A
:103EC0005B8D9380064B0022188803F075FF3FB08E
:103ED00000BDC046EA5BFF1FEB5BFF1F2C3BFF1FD3
:103EE000903CFF1FF7B50E00377A1C0008AB11009D
:103EF0003D001A8820231D401F423CD13378022BFD
:103F00003BD173681F785B781B023B431E4FBB425B
:103F100008D01E4FBB4214D01D4DAB4221D00A2504
:103F20002800FEBD002A2AD1142C2AD82200F068CD
:103F300007F0D6FC174B1C70012CF1D9FFF7B0FF2E
:103F4000EEE7002A1BD1202C1BD82200F06807F0D6
:103F5000C7FC114B04211C70104B187807F0D0FCE3
:103F6000DEE7E3B20124009201940A00310007F079
:103F7000AFFA0500D4E70825D2E70125D0E70B25E5
:103F8000CEE70D25CCE7C046F3FF0000F4FF0000AC
:103F900002290000EA5BFF1FC05BFF1F6C5CFF1F74
:103FA000332310B5040003700A220749013007F0DB
:103FB00097FC064B0F201B681A0AE37222731A0C37
:103FC0001B0E6273A37310BD345CFF1F5C5CFF1F8C
:103FD00030B5012503790400BFB02B4213D00B4943
:103FE000408806F0E1FD28420DD06A46084B02A841
:103FF0001B889380FFF7D4FF6B46D880002260882F
:1040000001A903F0D9FE3FB030BDC046E25BFF1FFF
:10401000863BFF1F10B5024804F050FD10BDC0469E
:10402000D13F001170B5160004AA148805AA1578AE
:104030004A685078117800022A4A084380180528F7
:104040004BD807F0CDFA03131E29343F0720032C69
:104050000BD80422121BAA4200D92A0022491A8036
:104060003000091907F03CFC002070BD0720112C1E
:10407000FBD81222121BAA4200D92A001B491A801F
:10408000EEE707200E2CF0D80F22121BAA4200D90F
:104090002A0017491A80E3E70720032CE5D80422F9
:1040A000121BAA4200D92A0012491A80D8E7072019
:1040B000032CDAD80422121BAA4200D92A000E4986
:1040C0001A80CDE70720032CCFD80422121BAA4266
:1040D00000D92A0009491A80C2E700220A201A8062
:1040E000C3E7C046DCD5FFFFAFBC0011085CFF1F73
:1040F0009FBC00119ABC001195BC001190BC00112E
:1041000010B50D21024A034806F0C6FC10BDC0469A
:1041100084BC00119C3BFF1FF0B50024274E85B0E6
:104120003000B47100F0E2F8254D264BEA89297C75
:104130009A422FD10423300003AA00F057F904005B
:10414000300000F011F90123B371002C34D16B461B
:1041500099892B68C9BA4B4329891B4A1B145B18E0
:1041600053806B46D9896B6849BA89B24B436989D8
:104170001B0C5B181548191C1BB2834200DD011C87
:104180000B0400D500211388918001331380200097
:1041900005B0F0BD0227220003AB3000009700F00D
:1041A000F7F80E230400297C0122300000976B44AD
:1041B00000F0EEF80443C3E71C00E8E7743CFF1F7F
:1041C0001C5CFF1F83050000345CFF1F0F270000ED
:1041D00073B5234E300000F089F8224D07236A465C
:1041E0003000297C00F002F904003000002C33D1AB
:1041F0006B461B787F2B2FD800F0B6F86B46D8782B
:10420000F02302041B031A406B469B8816495BBAD5
:104210009BB21A432B68000953432A891B0C9B1835
:104220004B806B465A789B7812031B011A436B68CC
:10423000024353436A891B0C9B180C481A1C1BB27F
:10424000834200DD021C130400D500220B888A8003
:1042500001330B80200076BD00F086F80124F9E7D9
:10426000743CFF1F1C5CFF1F345CFF1F0F27000006
:1042700070B5114C237C002B0FD0382B0ED10F4D75
:10428000280000F033F8CC23AC222800217C9B01CD
:1042900000F0F4F8280000F067F870BD084BE289E0
:1042A0009A42FAD1054D280000F020F8002228009B
:1042B000217C00F0C5F8EDE71C5CFF1F743CFF1F7C
:1042C0008305000010B5084B1A7C002A09D05B69F1
:1042D000002B06D09847041E01D0FEF791FE200067
:1042E00010BD0124F9E7C0461C5CFF1F70B5C17901
:1042F00005000C00631E9C411A4BE402E4184900BF
:104300000460C9B2007906F0D9F8E9796879490002
:104310000131C9B206F0D2F8E8790930C0B207F02D
:1043200087FA0023E36661332360AA795B3B002AA6
:104330000ED022689A43023B134323600A23E361B1
:104340000733236200232363A3630133E36370BD58
:1043500022689A4302231343236046236361063392
:10436000A361EFE70050004070B50025040003682A
:10437000DD66C0790930C0B207F0EAFB2900207978
:1043800006F038F82900607906F034F870BD0000B6
:10439000F8B51E0006AB1D78002304681700E3661D
:1043A000616007F035F901238022E3662B00276165
:1043B0005200013B08D207F013FB08200A4A11689B
:1043C000002D03D12800F8BD2261F2E7236F0342DC
:1043D00003D02369013D3370013613685B1A032B48
:1043E000EED90125EEE7C0466008FF1F70B51C003E
:1043F000002305681600EB66696007F009F90123E0
:104400008022EB6623005200013B08D207F0E8FA55
:1044100008200A4A1168002C03D1200070BD2A61CF
:10442000F2E72B6F034203D02B69013C3370013656
:1044300013685B1A032BEED90124EEE76008FF1F17
:10444000002370B504681500E366616007F0E0F8CA
:104450000123E366256107F0C3FA8020064A800045
:104460001168636B034205D113685B1A032BF8D9FB
:10447000012070BD0020FCE76008FF1F70B51D0023
:10448000002304681600E366616007F0C1F80123A9
:10449000E36626610F33626B1A42FCD02B0A23615C
:1044A0001023626B1A42FCD0EDB2256107F098FA36
:1044B0008020074A80001168636B034205D11368AE
:1044C0005B1A032BF8D9012070BD0020FCE7C04621
:1044D0006008FF1F70B51E00002305681400EB661E
:1044E000696007F095F80123A619EB660F33B44213
:1044F0000ED107F075FA80200A4A800011686B6BB4
:1045000003420CD113685B1A032BF8D9012070BD4C
:1045100021782961696B1942FCD00134E7E700205A
:10452000F5E7C0466008FF1F10B5084CE368002B94
:1045300008D1074B1B685B045B0C0A336360054BB7
:104540001B68236007F07CFAA06010BD5C5CFF1F55
:10455000C8F00040CCF0004010B507F059F80F4B00
:10456000996A9A6A8A42FBD10D4C6268A0688A18DF
:10457000121A531E884200D31300A1602168DA0B7F
:1045800052185B0407495B0C636022600B60064BAA
:104590001A6007F025FA206810BDC04600F0004000
:1045A0005C5CFF1FC8F00040CCF0004070B51F4CB1
:1045B00023793F2B01D93F2323711D4B22791A7098
:1045C0001878C0B207F034F818231A491A4A0B8039
:1045D0001A4913800B805380A379194980200B80DE
:1045E0000C21938001334B43164D191C000183426B
:1045F00000D9011C2980D1806379002B11D10133AE
:104600006371237A012B01D8022323726279237A02
:104610000D4853430A21584307F07AF90B4D28609F
:1046200070BDA02BEDD9A023EAE7C046505CFF1F68
:10463000480AFF1F8E3CFF1F5C3EFF1F8C3CFF1F84
:104640008A3CFF1F883CFF1F71020000405CFF1F77
:10465000F8B514210020FEF7C1FE114C011E114DCA
:1046600009D10C22104BC1CBC1C4280007F060F95E
:10467000FFF79CFFF8BD0C2220000C49FEF782FEDC
:104680000C2802D0084B43CB43C40C222800084915
:10469000FEF778FE0C28EBD00C220021E5E7C0469F
:1046A000505CFF1F1C5CFF1FF0BC0011FC0C0000E5
:1046B000F50C0000F0B51D4C8022A54404008820B4
:1046C00069465201400507F003F8902212016A443E
:1046D0001300200032C832C316C816C38023144CFE
:1046E000144FA6689B033343A3603B6007F018F99F
:1046F0008823A0685B05C01806F0CAFF0025882340
:1047000029008022A0685B05C01840196944520046
:1047100007F03EF880230135FF355B019D42EED165
:10472000A6603E60044B9D44F0BDC046FCEFFFFF19
:10473000D03DFF1F9808FF1F04100000F0B50400D3
:1047400087B0002825D0684607F012F91B4C0228D4
:1047500006D106226946200007F0B2F9002816D0DB
:104760006946002301250F262F00E25C0133100962
:104770001030874038002F00324097403A00024303
:104780004A610439062BEFD16846FFF793FF07B063
:10479000F0BD182269460A4806F09AFF6A46A3004F
:1047A000D358013305D01822FF21684607F0C0F81E
:1047B000EAE70134062CF1D1E9E7C0466509FF1F9D
:1047C00000090011F0B5002504000E0085B0AA42D2
:1047D00000D186E04B1C087801934B7889783779B3
:1047E00009021943F3783F061B040B431F43039749
:1047F00020706570252800D196E033D8112813D891
:1048000007F096F969002201220122012201AA0083
:10481000B800B1002201220122012201220122015D
:1048200022012201FC001C01232800D1D5E0DB2855
:1048300000D02BE1042A00D8ACE01025052A05D0D1
:10484000551F2A003800711D07F04AF80522310073
:10485000200007F045F82A003900601D07F040F8F5
:1048600005353EE0562859D010D8332800D19DE0B8
:10487000552839D02628DAD19A4B2900132218005E
:104880001D0007F055F8FEF7BBFB5CE0712800D176
:1048900077E0722800D180E0602800D18BE0DC282E
:1048A000C5D1022A00D875E07378BFB26370B378BF
:1048B000A370032A05D0033A390092B2F01CFEF728
:1048C0009BFC10223900E01CFEF75CFDC51C002893
:1048D00007DA60705CE00C222000834907F000F8E2
:1048E0000C25280005B0F0BD013A804D0C2A13D8E4
:1048F000002A0AD02800019906F0F2FFFFF756FEC1
:104900000C2228007A49FEF777FC29000C22601C53
:1049100006F0E6FF0D25E4E70C22EBE7734D754B3F
:104920002A0043CB43C2E9E7013A6E4D0C2A11D865
:10493000002A08D00199280006F0D2FF0C22280096
:104940006D49FEF759FC29001322601C06F0C8FFD0
:104950001425C6E70C22EDE705226849601C06F025
:10496000BFFF0625BDE712226549601C06F0B8FFAF
:104970001325B6E708226349601C06F0B1FF09253C
:10498000AFE77178F02905D85F4B188801F0B6FDC4
:104990000225A6E7FF236370FAE75C4B012A03D0E8
:1049A00072785A706270F3E75B78F4E72000FFF7E3
:1049B000F7FA050095E7013A554D082A0BD8002A69
:1049C00005D00199280006F08BFF01F06FF808224E
:1049D0002900601CD1E70822F3E7042A04D94D4DD1
:1049E0002F6007F02DF8A860FFF7B6FD04220390B2
:1049F00003A9601C06F074FF052572E7464D062AE0
:104A000015D906222800019907F05AF800280ED07F
:104A100006220199280006F063FF06223F4928007C
:104A2000FEF7EAFB0123394A51780B435370290002
:104A30000622601C06F054FF072552E7012AA9D080
:104A40007078FFF77BFEA3E7012800D0EFE6931E06
:104A5000334F1A2B04D87378002B09D100F014F9C6
:104A6000304B39001D78601C6A1E06F039FF38E7AC
:104A7000551E2A000199380006F032FF2A49AAB2D1
:104A80003800FEF7B9FB00F035F9E9E7DA281DD167
:104A9000042A00D87EE7082A15D9B37972791B0257
:104AA0001343F27912041A43337A1B0613433B6013
:104AB0003B68052231002000039306F011FF042219
:104AC000601D03A959E7FE236370F1E7DE2800D0DB
:104AD00060E7511E012A01D1002502E7019800F08C
:104AE000CBFFF9E71C5CFF1FFCBC0011505CFF1FF3
:104AF000FC0C0000F0BC0011F50C0000285CFF1F4E
:104B0000085CFF1FD43DFF1F903CFF1F4C5CFF1F44
:104B10002D3DFF1F5C5CFF1F6509FF1FADAC000052
:104B20004D5EFF1F4B5EFF1FAEDE000070477047FB
:104B3000020010B5094B0A32094C92B2DA815A824E
:104B400098811882207802F03FFB0422054B012156
:104B500020781A7006F0D4FE10BDC0465E3DFF1FDF
:104B6000965EFF1F955EFF1F013870B5042809D8B7
:104B700006F036FD030928081200234B022118789D
:104B800006F0BEFE70BD204B0821187806F068FEC6
:104B900000221E4B1A72F5E7802200241B4B1A4D8F
:104BA00052001A8108211A682878DC7206F0D8FEB3
:104BB0002100287806F07CFD012000F063FE00F063
:104BC00075FFDFE7104B0821187806F049FE104802
:104BD000FFF776F80F4B104A9B79002093800F4A1D
:104BE00013808022094B5200D8721A8100F04AFECD
:104BF00000F05CFF0A4B5B78002BC3D0094A1360BE
:104C000006F0D6FCBEE7C0466C5CFF1F405CFF1F91
:104C1000993CFF1F505CFF1F5C3EFF1F8A3CFF1F3B
:104C20004C5CFF1F34F0004010B501290BD1022865
:104C300009D1054B1B78002B05D02622034B0448D5
:104C40005A72FFF775FF10BD6E5EFF1F405CFF1FBD
:104C5000C40900000300F0B50A4D8E18B14202D11C
:104C600052008018F0BD0C782F6824093C5D0F2796
:104C70001C700C7801313C402F683C5D5C70023345
:104C8000ECE7C046843CFF1F0D22114B10B51A7093
:104C90000C23104C10492370093A033B0F486370F2
:104CA00006F01EFE2D2301220D490E48A371FFF7C9
:104CB000D1FF01220C49FFF7CDFF01220B49FFF77D
:104CC000C9FF00220A491000FEF796FA10BDC0463F
:104CD0006A5EFF1F4B5EFF1FAFBC00114D5EFF1FE2
:104CE0006709FF1F525EFF1F6609FF1F6509FF1F4F
:104CF000AEDE000070B5124C132220001149FEF701
:104D000041FB114D002817DDAB78002B14D0431C5C
:104D10002B7009236B700023001903702878290079
:104D20000130C0B206F06CFC297822000139C9B20A
:104D3000002005F0CFFD70BDFFF7A6FFEEE7C046EF
:104D40004D5EFF1FAEDE00004B5EFF1F10B5114B26
:104D50001A781870002A0ED000280BD10E4B1A7842
:104D6000062A07D85423D340DB0703D50B4B18780A
:104D700002F02AFA10BD0028FCD0074B1B78012B4B
:104D800002D0033B022BF5D8044B0121187806F022
:104D9000B7FDEFE76E5EFF1F955EFF1F965EFF1F7C
:104DA00070B54A4E4A4A4B493070022005F034FC37
:104DB00000F0E4FEFEF724F906F062FE0322464905
:104DC0004648FFF747FF2D24030004221C70444986
:104DD0000130FFF73FFF30230470424D424C4370D7
:104DE00083702E3B062220004049EB87FEF7CAFA6B
:104DF000062813D0200006F0BBFD022809D00321AD
:104E0000200006F0F5FC8D23E3706E3B237119330F
:104E10006371062220003549FEF7EEF9344B1B681A
:104E2000FC335C64FFF766FF0020FFF78FFF314C17
:104E3000314A0121314B1278207802F087F9304A4B
:104E4000304B12780021207802F080F901222E4B9D
:104E50001A702E4B9B78552B31D12D4B3B325A7209
:104E60002C4B2D4AAB81EA812B826A82202130783B
:104E700006F04EFE0120404205F078FD0120404240
:104E800005F014FEFFF73CF9FEF7FEFE00F0A4FC6F
:104E900001204042FEF7C6FF012006F079FEF02017
:104EA00001F010FB0121307806F02AFD307802F085
:104EB000E7FA1A4806F0CCFBFEF7FAFD70BD642253
:104EC000174B5B7953431A000A32CBE76C5CFF1F28
:104ED0002D4B0011294C0011D43DFF1F085CFF1F12
:104EE000285CFF1F5E3DFF1F6509FF1FADAC000082
:104EF000C85EFF1F965EFF1FB83CFF1F993CFF1F57
:104F00006A5EFF1F4B5EFF1F3C5EFF1F4C5CFF1F76
:104F1000405CFF1FC4090000CE0900006E5CFF1F4B
:104F2000505CFF1FF8B50A0020230D001A401942FB
:104F300057D0574B1B78002B50D0FFF70DFB554B2C
:104F4000554C564E99686268737A8A1ADB039A4206
:104F500002D36160FEF7ACFD327A217A531EDBB2D8
:104F6000994205D1FFF784F9002000F0D9FD0FE048
:104F70009142F9D300232372FFF7A4F9012000F036
:104F8000CFFD474F3800FEF79BFE390006F080FC4E
:104F9000637A002B1FD0013BDBB26372002B1AD166
:104FA000404B9B78552B01D106F002FBE37A002B96
:104FB0000CD000233C4A3A4FE37213883800013387
:104FC0001380FEF77DFE390006F062FC64237079E1
:104FD0005843FFF7ADFD237A013323722020684048
:104FE000F8BD0BB2002B0ADA304B187806F068FCDB
:104FF000002801D006F094FB80200002EFE7022495
:10500000214206D0244B01201A72FFF79FFE200098
:10501000E5E70B071ED5FFF79FFA1E4B1E491F4CF5
:1050200098684A68637A821ADB039A4202D348601E
:10503000FEF73EFDFFF746F9FFF71AF9012000F0F1
:105040006FFD00F0E3FB2368DB0701D5FEF7E2FF0D
:105050000820C4E71024214206D00D4B1B78002BFA
:10506000D5D1FEF725FED2E70124214207D0104812
:1050700000F06CF806F09CFB00F034FDC7E7042458
:10508000080020402142ABD0FEF7E8FEBFE7C04653
:105090006E5EFF1F5C5CFF1F405CFF1F505CFF1FCC
:1050A000993CFF1F4C5CFF1F345CFF1F6C5CFF1FB3
:1050B0007C3CFF1FF0B51B4B1B4F1B883A8804003C
:1050C0001A4E1B4D85B09A420DD832889A420AD3A7
:1050D000184B1A882B889A4205D1174A174B128809
:1050E0001B889A421BD0052001F042FA3B8802AA95
:1050F00013803388019053802B88114D93800F4B80
:1051000002A91B88D3800F4B2A78188802F05EFF13
:105110000D4B08212878019A1C7006F031FC05B06F
:10512000F0BDC0463A5EFF1F8E3CFF1F8C3CFF1F48
:105130008A3CFF1F385EFF1F365EFF1F883CFF1F43
:10514000965EFF1F903CFF1F345EFF1F13B50C4B94
:105150001C78002C11D1002801D00A4B18600A4A93
:105160000A4B11780A4A10780A4A01920A4A0092B8
:10517000002205F0A7FA200016BD1124FBE7C04667
:10518000955EFF1F305EFF1F945EFF1F845EFF1F52
:10519000965EFF1F705EFF1F745EFF1F10B5064B0B
:1051A00012201B78052B06D1044B13221988044BBF
:1051B000187801F0B9FB10BD955EFF1F903CFF1FF2
:1051C000965EFF1F10B500240122114B5242187049
:1051D000104B1C70104B1A8002F052F904220F4B36
:1051E00021001A700E480C3206F08AFA10222100B3
:1051F0000C4806F085FA07220B4B1C600B4B1C7009
:105200000B4B1C700B4B1A700B4B1C7010BDC04627
:10521000965EFF1F955EFF1F903CFF1F945EFF1F71
:10522000845EFF1F745EFF1F705EFF1F4A5EFF1FDC
:10523000495EFF1F923CFF1F485EFF1FF8B5174CE9
:105240000600257806A814240078052D23D1B41F64
:10525000134FA5B21824BD421DD88D1FADB2BD425B
:1052600019D8FA256D00AA4215D21D000D4F0A3D2E
:10527000ADB2BD420FD80C4C26800C4C21800C499D
:1052800000240A800B4A1380FFF714FF0A4B042105
:10529000187806F0E5FA2000F8BDC046955EFF1FBD
:1052A000790C0000750C00008E3CFF1F8C3CFF1F2A
:1052B0008A3CFF1F883CFF1F965EFF1FF0B50BB2B4
:1052C0000D0089B0002B00DB70E1A44E307806F0B1
:1052D000F7FA041E50D00378A22B00D122E1D02B84
:1052E0001AD0912B45D143780E2B42D19C4B82880A
:1052F0009A423ED19B4A83681278052A39D103200D
:1053000018567F2835D0984B1B68002B31D05B682E
:10531000002B2ED098472CE08078072829D806F05B
:105320005FF90428183F3F74A8D86378002B0CD18C
:1053300001218C4B19708D4B1A78002A5BD08C4B55
:10534000307801F003FF002855D00722854B1A70F2
:1053500051E061780029F8D1E378002B11D0854A1B
:10536000854B1278307801F0F1FE60706378002B85
:10537000EBD1200006F0D4F980200002684009B08B
:10538000F0BD784B1B78022BF3D00121307806F06A
:10539000FFFA0028EAD10121307806F0B1FAE5E7FA
:1053A0006378002BD1D16F4F032807D13B78052BB1
:1053B00002D101333B701EE00223FBE76F4B1A88DA
:1053C0006F4B0293002A0BD01B78002B03D00121D6
:1053D000307806F0D5FA3B78062B04D1013BE9E79B
:1053E000029B1A70F7E7042B41D10121029B307810
:1053F000197006F085FA5C4B1B68002BB9D01B684E
:10540000002BB6D0574A107884E76378554F002BAD
:1054100027D10622211D5B4806F062FA62895A4BA9
:105420005A491A80A2895A4B1A80E3890B800521B8
:10543000397058490A80584A1380228A574B1A807B
:10544000574B1B78012B09D11F2001F091F8FA224C
:10545000920042430421307806F092FA0022484B31
:1054600075E7312B00D070E70022454B1A700323FB
:10547000A0E706220021434806F042F90023454AEE
:1054800004211380444A30781380444A138006F084
:10549000E7F90821307806F0E3F9A379083B5A428E
:1054A0005341304A03331370304B1B78002B06D026
:1054B000334B30781A78002A06D001F085FE01229D
:1054C000314B52421A8096E70121197006F018FA02
:1054D000F5E70821307806F0C3F96378002B00D097
:1054E00047E72C4B2D4F0293E388029A0421138047
:1054F000294B307803932389039A138063893B8077
:1055000006F046FA002800D033E7264B1B68002B34
:1055100000D12EE7039902983A88098800881B6811
:10552000984726E74379132B00D022E70389012B04
:105530000AD11D4B1B78022B06D10821307806F0CA
:105540008FF9FFF72BFE14E7052001F011F8082171
:105550000200307806F014FA0BE7C046965EFF1F93
:1055600005140000955EFF1F305EFF1FB83CFF1F53
:10557000993CFF1F6A5EFF1F4B5EFF1F6C5EFF1FA3
:105580006E5EFF1F3D5EFF1F903CFF1F445EFF1FCE
:10559000465EFF1F3A5EFF1F385EFF1F365EFF1F2D
:1055A0003C5EFF1F2C5EFF1F345EFF1F8020C0018A
:1055B000014200D0E2E6CB0731D5324B1B78002BFD
:1055C0001DD0314E05AC3378052B1AD1023B237028
:1055D0002E4B21001B7823722D4B1B7863722D4BB1
:1055E000187801F057FD002809D007202A4B3070A9
:1055F0001B68002B03D01B68002B00D098470120AC
:10560000BCE60E20254B06221B7825492370254B2E
:105610001B78637002ABC01806F062F9D8E702236A
:1056200008001840194209D0174B1B78052B03D1ED
:105630001D4B188806F0BCFA02209FE60424214284
:1056400003D0FFF737FD200098E608230800184034
:10565000194200D193E6154B1C78012C03D0022C83
:105660000DD008208AE6124B124A134913481B88B2
:105670001288098800880094FFF7E0FDF1E7FFF742
:105680008DFDEEE76E5EFF1F955EFF1F923CFF1FD4
:10569000485EFF1F965EFF1F305EFF1F4A5EFF1FC2
:1056A000933CFF1F495EFF1F903CFF1F345EFF1FAE
:1056B000883CFF1F8A3CFF1F8C3CFF1F8E3CFF1F56
:1056C00010B502A804880B20002C10D14968087876
:1056D0004978090201430C48814209D1022119800D
:1056E0000A4B59881170DB7800205BB2537010BDF3
:1056F000074C0A20A142FAD102211980034B998854
:1057000011705B79F0E7C0466E2A0000345CFF1F21
:105710006F2A0000F7B5150008AA16884A680F4FCF
:1057200014785278120222430A24BA4214D1012278
:10573000DBB2019200962A0005F0CAFE041E0BD1CE
:10574000074B1B68002B07D068782A7800021043AB
:1057500042425041013098472000FEBD022900001E
:10576000A85EFF1F30B5012503790400BFB02B42AE
:1057700025D01449408805F017FA28420CD0124B66
:1057800001A95B8D00220B8002234B800F4B5B88AD
:105790008B80608802F010FB0D49608805F004FAE8
:1057A000C0070CD50B4B01A91B8800220B800223DC
:1057B0004B80064B9B888B80608802F0FDFA3FB0DF
:1057C00030BDC046A05EFF1FBC3CFF1F345CFF1F06
:1057D000985EFF1F163DFF1F10B5074C07492000BC
:1057E00005F098F92000064905F094F90721054ACB
:1057F000054805F051F910BDFFFF0000A05EFF1F36
:10580000985EFF1F1CBD0011BC3CFF1F10B5024875
:1058100003F054F910BDC04665570011082110B5BA
:105820000E240A4AC307DB170B405179A1430B43EF
:1058300053710223184202D051790B435371042350
:10584000184202D051790B43537110BD2D3DFF1FFB
:105850000A2110B50F240A4AC307DB170B40117841
:10586000A1430B431370830703D5062311780B4321
:105870001370400703D5012311780B43137010BD3B
:105880002D3DFF1F10B5054B102419780A00A243C7
:10589000002801D022000A431A7010BD2D3DFF1FC1
:1058A000662110B52024134BDA788A431979DA700F
:1058B000A14324190C431C71542812D960200143C0
:1058C000197104210A43DA700222D9780A43DA7086
:1058D0002022D9780A43DA704022D9780A43DA7054
:1058E00007E04428EDD83428EED82428F0D814282E
:1058F000F2D810BD2D3DFF1FF8B50E23384C050022
:10590000627926791A4011339E43364B62712671B3
:10591000984204DD6E23E3716C3BA371F8BD324BFA
:10592000984203DA1A23E3711C33F6E700232F4968
:10593000A371E37183B259182D4889B2814224D9E9
:10594000681D0A2100B205F0E3FF2A4B00B29D4218
:1059500044DC05006421280005F0DAFF0A2100B2CA
:1059600006F00EF9244F09B2E2797B5C1343E37130
:105970000A21280005F0CCFF0A2100B206F000F948
:105980001D4F09B27B5CA2790EE001210A436271CE
:10599000002D1CDA5B421DB20423A371A379632D91
:1059A000D8DCFA22092DE3DC1343A3710A21280075
:1059B00006F0E6F80F22114F09B27B5C1A4016433D
:1059C0001F2293436279267113436371A6E7FA237A
:1059D0009B009D42E2DB0123E371BBE70500FAE790
:1059E0002D3DFF1F1B4E00001DFCFFFFCB070000DD
:1059F000960F00000A27000066BD001156BD001179
:105A000070B51B4D04002B7900290DD08022134363
:105A10002B71632C0BDD76236A7813436B70402364
:105A2000AA781343AB7070BD7F221340F0E72300C8
:105A3000093306DA58236A7813436B70AA786C230B
:105A4000EFE70C4E002C0ADA2023644224B26B707C
:105A50000A21200006F094F809B2735CE2E7092CF1
:105A6000F6DD0A21200005F053FF00B2335CEEE7BB
:105A70002D3DFF1F46BD0011F8B50A4F05003B78CC
:105A80000E00002B0CD0084C2000FEF72FFC33003A
:105A90002A0020003978FEF71DFD2000FEF764FC87
:105AA000F8BDC046B55EFF1F383DFF1F70B50A4EFA
:105AB0000A4D08223100280006F002F8002809D01B
:105AC000074C31000822280005F00AFF09212000B8
:105AD000FFF7D2FF70BDC0462D3DFF1FAD5EFF1F1B
:105AE000AC5EFF1F102110B50C4B36201A78987150
:105AF0000A401A70DA7856310A40DA706022197951
:105B000098701140223ADA71A2325A71DF3A0A4390
:105B10001A7106225A70FFF7C9FF10BD2D3DFF1FF5
:105B200010B5002824D0134C0A210223E05E05F0B2
:105B3000EFFE00B2FFF7E0FE0423E05E642105F013
:105B4000E7FE012100B2FFF75BFF207AFFF7A8FE16
:105B50000320FFF763FE0020FFF77AFE064B18785C
:105B6000053843425841C0B2FFF78CFEFFF79EFF55
:105B700010BDC046345CFF1F955EFF1F70B5002549
:105B80000A4C2000A571FEF7B1FB10233E21200036
:105B9000074AFEF79FFCA84200D13E35054B200086
:105BA0001D70FEF7E1FB0123A37170BD383DFF1F9F
:105BB00036BD0011B55EFF1F0200F0B501270A488F
:105BC0000A4E51188B1A002B00DCF0BD0824157802
:105BD0004308684038404000805B013C58406D08F5
:105BE000002CF5D10132EDE7FFFF000076BD00117A
:105BF000F0B500250F269D4200DBF0BD4C5D070986
:105C000044403440A400A05801357840F3E7000038
:105C1000F0B589B06A460D000B000F271100103552
:105C20001C780133260024093E401670547002325D
:105C3000AB42F5D12023024AFFF7DAFF09B0F0BDED
:105C40007CBD0011F0B54E780B7889B036020C009F
:105C5000170001901E43012A61D9954B9E4200D83E
:105C600077E001339E421CD1062A17D1CA788B787F
:105C700012021A430B791B0413434A7912061A4382
:105C80008C4B5A6100221A705A808B4A5A608B4A98
:105C90009A608B4ADA60002009B0F0BD8822520574
:105CA000EEE7884B9E423CD182498B78002B00D096
:105CB000F6E00C2A31D10F22A3789343E278120246
:105CC00013432279120413436279120613434B6083
:105CD000E279A07912020243207A00041043627A2A
:105CE00012060243CA60E27AA07A120202437648A0
:105CF0004A81834208D804236E49142201980B700C
:105D000005F0EEFD1420C7E71201D21889235B05C8
:105D10009A42F0D801238B70BDE7022AFAD00523FE
:105D2000EAE76A4A01239642E6D1FFF737FA052FE0
:105D30000CD9E378A2781B021343227912041A4388
:105D400063791B061343624A0393136005F030FC2A
:105D5000A1E7584D2B78002B9DD1AB78002B00D1BB
:105D6000A0E02B8901339BB20093B34200D091E0B5
:105D7000132AD4D9CF7C8B7C3F02122120001F43F1
:105D8000FFF71AFF874200D08EE0002E3DD1E37866
:105D9000A2781B0213432279E96812041A4363793B
:105DA0001B06134303930A228B4212D1FF23A370D5
:105DB000E370237163716B89002B09D1E37B227C33
:105DC0001B0212041343A27B13431B0901336B8193
:105DD00000226B89002B8ED0002A67D168683701BA
:105DE0003818000B6B6900030390984205D968616D
:105DF00005F04EFCEB780133EB7068681022A11CB3
:105E0000381805F0C5FC2E8145E76F89009A7B1E86
:105E10009BB293423AD1E278A37812021A432379D3
:105E200005A81B04134362796C6812061A43EB68D9
:105E300000920392211D0C22049305F051FD0120D4
:105E4000260004A940421036FFF7E2FE013F012F71
:105E500017D1009A0B232861824200D04CE704221C
:105E60001C49200005F094FC042203A9686805F091
:105E70002FFCE968039AFF23914200D13CE7F73BEE
:105E80003AE73100FFF7C4FE1036DFE70923B742D7
:105E9000A4D831E7009BB34200D9FCE607232BE7E7
:105EA000022329E7032327E7062325E70A2323E71D
:105EB000FFFE0000403DFF1F00000111FFFF00003A
:105EC0005048593601FF0000FFFF001102FF00009B
:105ED00034F000404C3DFF1F10B5034C0B00012275
:105EE000210000F06BFA10BD996000110B8870B5AD
:105EF00006000D000224162B11D92B00032209499C
:105F000000F05CFA041E0AD1074B2A881B88191C72
:105F1000934200D9111C300089B200F0EFFA200042
:105F200070BDC046C5600011E25EFF1F10B54A7823
:105F30000400013A0B000220012A07D80A78002A3F
:105F400004D005222000024900F038FA10BDC046F6
:105F5000F36000110A7810B50B0004000220002A3B
:105F600004D007222000024900F028FA10BDC046E4
:105F70009F6100110A7810B50B0004000220002A6E
:105F800004D009222000024900F018FA10BDC046D2
:105F90000562001110B5034C0B000B22210000F02C
:105FA0000DFA10BD3562001110B5034C0B000D2227
:105FB000210000F003FA10BDA762001110B5034CD8
:105FC0000B000F22210000F0F9F910BD0163001150
:105FD0000A7810B50B0004000220002A04D0112218
:105FE0002000024900F0EAF910BDC046116300111B
:105FF000002310B51322190000F0E0F910BD0000D5
:1060000010B5034C0B001722210000F0D7F910BD8A
:1060100063630011002310B51922190000F0CEF9B6
:1060200010BD000010B5034C0B001B22210000F036
:10603000C5F910BD9D630011F7B584890D000600F8
:106040000121002C22D000238268D3561778002B20
:106050001EDA0C2C1AD90C3CA4B2131940880093F8
:10606000230002F086FE431E984101307B06DB0FC1
:106070006B703F23013C1F40A4B22870AF70AC800E
:10608000002C07D0B3680133AB6000210800FEBDCF
:106090000020EBE7AC60F8E70B7803704B884370A7
:1060A0004B881B0A83700B79C3700420704704204F
:1060B000022B06D10020537811781B02009A0B4363
:1060C000138070470B8803700B881B0A43700220F3
:1060D00070470420009983420AD1537810781B023C
:1060E00003430B80D37890781B02034300204B803E
:1060F0007047F8B50D004B7801240021461C037051
:106100002B788B4201D82000F8BD6B78B01C4F1C57
:10611000012B10D1890069184B88022233704B88FB
:10612000B9001B0A7370691805F0C2FB0436043409
:10613000A4B2F9B2E4E7122359436B185A88043128
:1061400032705B8810221B0A7370691805F0B0FB6F
:1061500012361234ECE770B5049D14001E00052BB6
:1061600001D8042070BD637812781B0213432B8082
:10617000E378A2781B02134302226B802A71211D4F
:10618000681D063E05F094FBB2B22A81E92AE8D8E0
:106190002800A11D0A3005F08BFB0020E2E7002358
:1061A00010B50A789A4201D8900010BD9A008A185A
:1061B0005488013304705488DBB2240A44709488F4
:1061C00084709288120AC2700430EAE710B5110098
:1061D000029C062B04D004201022142B01D010BDE9
:1061E000022222714B7808781B0203432380CB786C
:1061F00088781B02034363800431601D05F058FB5F
:106200000020ECE710B50C788B7804315C43E4B2E5
:1062100003702200013005F04BFB601C10BD042010
:10622000022B06D10020537811781B02009A0B43F1
:106230001380704710B50C000A88023105F038FB56
:10624000208810BD70B504000D0004981100012BCA
:1062500001D8042070BD16785278120232430280B1
:106260000200F13255701470E125002C00D10C357C
:10627000023B9AB24280AA42EBD80231043005F0C8
:1062800017FB0020E6E70420009983420AD15378E7
:1062900010781B0203430B80D37890781B020343D2
:1062A00000204B80704710B50C000A88023105F0C1
:1062B000FFFA208810BD000070B501211E000420E7
:1062C000049C0E400B4218D1CB40DDB28D4214D954
:1062D0000A49DBB2098899420FD32300EE331D70BF
:1062E0003300580011184978165C09023143013314
:1062F0002152D9B28D42F4D8002070BD583DFF1F05
:1063000010B50C000A88023105F0D2FA208810BDC1
:1063100010B50C788B7804315C43E4B20370220032
:10632000013005F0C5FA601C10BD10B511000298CF
:10633000032B01D8042010BD14785278043B1202BC
:1063400022430280CA788C781202224342809AB299
:106350008280EB2AEED80431063005F0A9FA00203D
:10636000E9E710B50C000B8803700B881B0A43701B
:106370004B8883704B881B0AC3708A8804300631AF
:1063800005F096FAA088043080B210BD0420012BDD
:1063900003D100201378009A1370704710B50C00D9
:1063A0000B8803700B881B0A43704A880230043143
:1063B00005F07EFA6088023080B210BDF0B589B079
:1063C00003931E4B029242000700D05A019102F043
:1063D00020F81325061E2DD0029B01240370019B7B
:1063E000002B04D0001903999847001984B26B461A
:1063F0001B7A5BB2002B0FDA1021380002F01CFB75
:106400001925002813D130003219E1B202F066FCE0
:10641000051E0CD10C34A4B2042304AA380005A92B
:1064200093800696948101F0AFFD051E02D03000E6
:1064300005F006F9280009B0F0BDC046E05EFF1F78
:1064400070B505000C0000280CD00020814209D056
:1064500010222000044905F02BFA01202B78237329
:106460006B78637370BDC046BCBD0011F0B506000B
:106470000D0017001C0085B002291BD00020102938
:1064800007D1022B07D0102B03D115E00020102CD0
:1064900008D005B0F0BD69463800FFF7D1FF2A00EB
:1064A00069460BE069463000FFF7CAFF22006946E3
:1064B000380004E0022BE9D12A003900300005F051
:1064C000AFF8E6E7031CF02800D9F02303200849C1
:1064D0009AB2013A0B80D317034006499B189B10D0
:1064E0000B80D30F04499B185B100B807047C0468C
:1064F0005C3DFF1F5A3DFF1F583DFF1F034B1B888C
:106500008B4202D3024B4000C15270475C3DFF1FDB
:10651000E05EFF1F014B4000185A7047E05EFF1F0E
:106520001722014B1A807047E05EFF1F70B505000F
:106530000E2005F05DF8041E13D0D0230370002355
:106540000622837007494570033005F0B1F9064B08
:106550002100DA8A62811B7E2373044B187805F0D0
:10656000F7F970BDFC5EFF1FEC5EFF1FAC3DFF1F27
:10657000262803D8024B4000C05A70470148FCE768
:106580005E3DFF1FFFFF000070B506000C00094DC7
:106590001C220021280005F0B3F8074B1E70074BA2
:1065A0001C7005F0FDF90123002801D00023122002
:1065B0002B7070BDEC5EFF1FAC3DFF1F0D5FFF1F1A
:1065C00070B505000D4C0800E260A16010220021AA
:1065D000656005F0F5FA012803D11021A06802F0EA
:1065E00058FD10220021280005F0EAFA012803D105
:1065F0001021606802F04DFD70BDC046EC5EFF1FCB
:1066000070B5041E05D1002903D006220D4805F0FF
:106610004FF90D4B1D78012D11D1002C05D102220F
:106620001A7005F055FA280070BD00221A70074B49
:106630001B78FF2BF7D02000FFF778FFF3E700254A
:10664000F1E7C046FC5EFF1FEC5EFF1FAC3DFF1F85
:10665000030010B5002801D1002010BD00780B4ABE
:10666000002803D15988D1821B7913761378022B25
:10667000F2D10023984200D103331370044B1B78EE
:10668000FF2B01D0FFF752FF0120E6E7EC5EFF1F72
:10669000AC3DFF1F002911D000280CD04B790128F8
:1066A00003D140225242134303E03F221340032808
:1066B00002D001204B7170474022F4E70800FAE74E
:1066C00070B5094D0100287800280BD0074C062230
:1066D000200005F0EDF821002878FFF7DBFF20000F
:1066E00005F0F6F870BDC0460C5FFF1FE65EFF1FA9
:1066F00000290AD0012808D13F224B799343C02BAF
:1067000003D0403B5A425341981C704770B5174D17
:1067100006002B78FF2B15D00A2004F069FF041E19
:1067200010D0D0230370C83B8370114B11491B78E4
:106730004670C3700622043005F0BAF821002878AC
:1067400005F006F90C4B1B78012B0DD10B4B1B6888
:10675000002B03D09B68002B00D09847084B0421E6
:106760001878084A05F0FCF870BDC046AC3DFF1F24
:106770000C5FFF1FE65EFF1F085FFF1F345FFF1FF8
:10678000385FFF1F60EA0000014B98687047C04601
:10679000EC5EFF1F014BDB6818687047EC5EFF1F63
:1067A000074B10B5DA68136801331360054B18788E
:1067B000FF2803D08021C90105F0A2F810BDC04612
:1067C000EC5EFF1FAC3DFF1FF7B50E0002F0C8F8EE
:1067D000051E1CD00E4B06621F78002F00D10778D3
:1067E000AB791020019304F003FF041E0FD0D023D7
:1067F0000380C73B8370019BE91DC37006220430F0
:1068000005F056F821003800E66005F0A1F8F7BD64
:10681000AA3DFF1F014B18787047C0460C5FFF1F51
:10682000054B002805D1054B1A78054B002A00D1ED
:10683000014B18007047C046FC5EFF1F0C5FFF1F36
:10684000E65EFF1F014B58687047C046EC5EFF1FB5
:10685000024B1868431E9841C0B27047105FFF1F7B
:10686000421E03000120152A03D9FF3B5A4253411F
:10687000D8B27047F0B51C0000230E0085B003901D
:1068800002920B70029A934201D3002019E0E55C5A
:106890005A1CD2B2002DF8D0029851198142F4DC72
:1068A0000233DFB2A35C18000193FFF7D9FF002881
:1068B00007D0013D019A0399EBB233708A4202D1AD
:1068C000E01905B0F0BDDB19DBB2DBE710B50C0059
:1068D00002F09EF803001220002B03D021005888FC
:1068E00005F0DEF810BD000070B50E4D8400635950
:1068F000002B15D0186A002801D004F051FF2B5945
:10690000586A002801D004F04BFF2B59986A0028E0
:1069100001D004F045FF285904F042FF00232B5119
:1069200070BDC0461C5FFF1F1C4B70B504000E00FD
:10693000150099420AD11A4B1B68002B01D1122075
:1069400070BD1B68002BFAD09847F9E7154B9942A8
:1069500015D1134B1B68002B0AD01B68002B07D0E6
:106960009847002804D1104B1C70104B1D70E7E7AE
:1069700029002000FFF7AAFF0028E1D1F3E7080073
:1069800001F0EEFF0028DAD003780320A342D7D12C
:106990002900300005F084F8D2E7C046FEFF000071
:1069A000185FFF1FFFFF0000155FFF1F145FFF1F31
:1069B000F7B50400808801F0D3FF0025A84203D07A
:1069C0000578A08802F008F81C4E3378002B1FD001
:1069D000AB421DD11A4B28001978FFF777FF00282A
:1069E00018D000233370A3790820A778A6880193D4
:1069F00004F0FEFD011E0DD0D0230370CA3B83704E
:106A0000019B477086808371280004F0A1FF01E09C
:106A1000002DE8D1A0880B4B8200D358002B01D069
:106A2000FFF762FF1721A088FFF768FDA08801F03B
:106A300027FDA08801F0FEFDF7BDC046155FFF1FD2
:106A4000145FFF1F1C5FFF1FF0B587B01D000CAB6C
:106A50001B88070001930DAB1B88142002930EAB1B
:106A60001B88160003930FAB1B880091049310AB97
:106A70001B88059304F0BCFD041E1AD0D0230370BC
:106A8000CB3B47708370C670062229000430002D6E
:106A900011D004F00DFF019B21006381029B00983F
:106AA000A381039BE381049B2382059BA37404F0D1
:106AB0004FFF07B0F0BD04F023FEECE7F7B50093FD
:106AC00008AB1B8807000C200D001600019304F092
:106AD0008FFD041E13D0280001F042FF00280FD0C4
:106AE0000078D0232370C93BA370009B2100238131
:106AF000019B6770A580E680638104F029FFF7BDE4
:106B0000014B1878EDE7C046AC3DFF1F13B50400FC
:106B100064890389C2888188C0780094FFF7CEFF1A
:106B200013BD000010B5044C2068002803D004F009
:106B300037FE0023236010BD205FFF1FA122F0B5A8
:106B4000818892004A43384B384F1B6804009B18D9
:106B50009D2292009B18827989B01A603B68002BB5
:106B60005FD01D78324B1B68002B04D05B68002B74
:106B700001D000209847260008363100E079FFF761
:106B8000B7FD237DE0710200E0780493638A290059
:106B90000393238A0293E3890193A388009333002C
:106BA000FFF752FFE378002B0BD1E289A379A1888C
:106BB00002920196E27928000092012201F0DAFEA9
:106BC000E0703B68002B20D0FFF7ACFF194D287810
:106BD00000281AD0184B1978FFF778FE002814D037
:106BE0002B78E67808200793A78804F001FD011EA2
:106BF00009D0D0230370CA3B4670837087808671AA
:106C0000079804F0A5FE00232B701721A088FFF73A
:106C100075FCA08801F034FCA08801F00BFD09B0E0
:106C2000F0BD064B9DE7C0463409FF1F205FFF1FE4
:106C3000345FFF1F155FFF1F145FFF1FAC3DFF1F79
:106C4000F8B5070008000E0001F08AFE041E18D0F7
:106C50002620FFF78DFC051E00D12578062004F0C4
:106C6000C7FC041E0DD00021062204F049FDD023EC
:106C70002370C23B21006770A370A680E8B204F0C5
:106C800067FEF8BDF0B585B001930AAB1B7807002D
:106C900002930BAB1B7808000D000092039301F0E8
:106CA0005FFE061E22D0102004F0A2FC041E1DD0A0
:106CB0001022002104F024FD2620FFF759FC0028B3
:106CC00000D13078D0232370C13BA370009B2100FA
:106CD0002372019B67706372029BA580A372039B62
:106CE000C0B2E3720C9BE36004F032FE05B0F0BD6D
:106CF000F7B50D00019001F033FE071E20D00E20E5
:106D000004F076FC041E1BD02620FFF731FC061E83
:106D100000D13E78D0232380C53B0622A370F91D05
:106D2000E01C04F0C5FD019B2A0063810123DD40C6
:106D30001A401D40210022736573F0B204F008FE72
:106D4000F7BD0000F0B585B0029010000D001700EF
:106D50000A9E039301F004FE041E31D0029B002B17
:106D60002ED1039B02795B0724D5122313430422FF
:106D7000002E08D10B99002905D10C99002902D1C8
:106D80000D9900291AD01A430D9B2271002B00D0B7
:106D9000C9E0002E00D1CFE0002D00D0CCE0606A29
:106DA000002801D004F0FCFC1C21300004F070FE2F
:106DB000606205E002239A430E33D7E793432371C1
:106DC000654BBA00D458002C00D1AAE0002E10D098
:106DD000236A002B03D11C2004F0E2FE20625E4BEC
:106DE000BA00D358186A002803D01C22310004F0DE
:106DF0005FFD0C9B002B12D0574CBB001D596B6ADA
:106E0000002B03D1162004F0CBFE6862BB00E358D0
:106E1000586A002803D016220C9904F049FD0D9BF6
:106E2000002B11D04C4DBC006659B36A002B03D126
:106E3000142004F0B5FEB0622B59986A002803D0E4
:106E400014220D9904F034FD380001F089FD051E6F
:106E500067D0414BBA00D358002B62D01A6A342055
:106E6000002A00D11C389A6A002A01D0143080B25E
:106E70000B9A002A01D01C3080B25B6A002B01D033
:106E8000163080B204F0B4FB041E4AD01822002150
:106E900004F036FC2620FFF76BFB0190002801D19F
:106EA0002B780193D0232370029B200063700A2368
:106EB000294EA370039BBD00A371AB59A780196A2B
:106EC0001830002905D01C22A06004F0F1FC20003D
:106ED00034307359996A002907D0030014221433FF
:106EE000E060029304F0E4FC02980B9B002B08D0B6
:106EF00003001C221C330B992061029304F0D8FC80
:106F000002987359596A002903D01622606104F06F
:106F1000CFFC6B462100187904F01AFD3800FFF70A
:106F2000E3FC05B0F0BD10220D9B0D991B69A01864
:106F3000236204F0BDFC2CE70B9B002B00D13FE744
:106F4000012D00D03CE7606A002801D004F028FC45
:106F50001C210B982AE7C0461C5FFF1F10B5044C8C
:106F60002068002803D004F01BFC0023236010BD20
:106F7000105FFF1F0B4B07B51A68002A01D10020D4
:106F80000EBD6946531C012012780731FFF772FCD1
:106F90000028F4D002780123100018401A42EED0E5
:106FA000EEE7C0462C5FFF1FF0B51F4F01203B6886
:106FB00087B0002B25D09B78059300F0B3FB002809
:106FC00021D00A20FFF7D4FA04000B20FFF7D0FAF3
:106FD000164B05001E78731E9E413B68F6B2191DC4
:106FE000D878FFF757FB3B682900DA7A043303921D
:106FF0009A7901930292009033002000059A04F0E0
:107000000FFC07B0F0BDFFF7B5FF002805D0062044
:10701000FFF7AEFA04000720D8E70820FFF7A8FA28
:1070200004000920D2E7C046105FFF1F0C5FFF1F5E
:1070300070B50A4E040033780D00FF2B0DD00420EC
:1070400004F0D6FA011E08D0D0230370CE3B457061
:107050008370C470307804F07BFC70BDBC3DFF1FB2
:1070600070B5040006200D0004F0C2FA011E0AD01B
:10707000D0230370CD3B8370054B44701B68858023
:10708000187804F065FC002C01D0FFF767FF70BD95
:10709000105FFF1FF8B5264F06003B680D00112456
:1070A000002B05D10522234B1B78134202D1122459
:1070B0002000F8BD204A10241268002AF8D0127867
:1070C000002AF5D0DB0719D52B789A1E012A1AD889
:1070D0000C2004F065FD132438600028E8D000235C
:1070E0000A22437029000670023004F0E1FBFFF72A
:1070F0005BFF041E0AD0FFF731FFD9E700F012FB57
:107100000028E1D1E4E7002BE2D0D0E70B4B1B785D
:10711000032BCDD11D20FFF72BFA094B1880002837
:10712000C6D0084B04211878074A04F019FCBFE7C1
:10713000105FFF1F0D5FFF1F2C5FFF1F0C5FFF1F06
:107140000A5FFF1F385FFF1F60EA0000F7B5019379
:10715000194B14001A78052306000F0012201A425A
:1071600021D0012920D1154B1D68002D1BD00220F4
:107170001F2C18D8002C02D0019B002B13D0104BD1
:107180001F221E706E1C0021300004F0B9FA019914
:107190002200300004F08CFB310020002C70002F06
:1071A00006D004F06DFBFEBD064B12201D68DCE727
:1071B00004F026FAF7E7C0460D5FFF1F2C5FFF1FA4
:1071C000BC3DFF1F285FFF1FF8B50F4E1224336828
:1071D000002B17D01B780F3C834213D100250B4F97
:1071E0000221387804F03CFB094B042138781D80DB
:1071F00004F036FB074B28001D8033685C7004F0F8
:10720000BFFA04002000F8BD105FFF1F385FFF1FAA
:10721000245FFF1F0A5FFF1F70B5012823D11B4C9D
:107220002388002B03D01A4A1578002D07D0194B5C
:107230001B68002B02D01878FFF7C6FF70BD3B2BF0
:1072400002D93C3B2380F9E7134E0221307804F049
:1072500007FBFA222388920002215A43307804F077
:107260008FFB2580EAE70B4B1B68002BE6D00B4B0E
:107270001B785B07E2D5084B0221187804F0F0FA7E
:107280000022024B1A80FFF769FED7E7245FFF1F39
:10729000085FFF1F105FFF1F385FFF1F0D5FFF1F9D
:1072A000F8B51E4D2868002803D004F079FA0023B1
:1072B0002B601B4E3068002803D004F071FA0023C5
:1072C0003360184F05243B7818002040234221D01A
:1072D000154800F02BFA3B78234213D0202004F00D
:1072E0005FFC2860002813D02022002104F008FA57
:1072F000202004F055FC041E306005D0202200211F
:1073000004F0FEF9002004E0286804F049FA2C603B
:107310001320F8BD00F00AFAF4E7C0462C5FFF1F07
:10732000285FFF1F0D5FFF1FB03DFF1F10B50A4C08
:1073300023681A1E0ED0002808D10130587004F0BE
:107340001FFA002805D02368002B02D00021FFF788
:1073500087FE0122100010BD105FFF1FF7B5274EFA
:10736000050033680191181E21D05C78244F012C50
:1073700030D1FFF7FFFD002825D02000FFF7F8F8F7
:107380000400412814D91F4B022118781E4A04F02A
:10739000E7FA1E4B3C3C1C80022233685A703B7853
:1073A000002B14D128000199FFF75AFE0120FEBDE1
:1073B000FA2292004243002AEED0124B02211878A2
:1073C00004F0DEFAE8E7FFF7D3F80200F3E7002362
:1073D0003B70EBE73B78002BE8D1032004F008F981
:1073E000011E08D0D0230370CC3B457083703368F6
:1073F000187804F0ADFAFFF7B1FDD7E7105FFF1F73
:10740000085FFF1F385FFF1F60EA0000245FFF1F57
:1074100010B51749838802008B4220D011D8154936
:107420008B4217D0144900205B1899B2012907D864
:10743000926811785A425341D8B2FFF7F9FD012002
:1074400010BD0E4A00209B1807229BB29A42404171
:10745000C0B2F5E783681878FFF768FFF0E7836844
:1074600099785A78090218781143FFF777FFE7E710
:107470000A20000006200000F8DFFFFFAFDFFFFF5B
:10748000014B18707047C046BD3DFF1F10B5064C3C
:10749000207001F041FA207804F02AFB05212078C1
:1074A00000F062FD10BDC046385FFF1F0BB273B520
:1074B0000D00002B00DBC4E0884B187804F000FAC4
:1074C000041E0ED00378912B0FD0A22B00D1A1E087
:1074D000834B1878FF2852D0210004F039FA002895
:1074E0004DD180200002684076BD43780F2B76D0C6
:1074F00013D8052B70D00E2BEAD18088794B984297
:107500002BD8794B98421BD8784B9842E0D1A3688E
:107510001878591CFFF774F838E03E2BD8D18378DF
:10752000032B74D06CD8012B6ED0022BD0D1704BB2
:107530001B68002B23D05B68002B20D098471EE0EF
:107540006C4BC0180C28C3D804F0AAF81DC2C21591
:107550000BC20B0B0B3223C23C00674BC018072831
:10756000B6D8664B1B68002B09D01B68002B06D0D1
:10757000200098470AE0A3681878FFF7C7F82000B2
:1075800004F0CEF8ADE7A068FFF762F800289FD0BE
:10759000F5E7A3681B78002BF1D0554B1B68002B37
:1075A000EDD01B68002BEAD0210055489847EDE745
:1075B0004F4B1B68002BE2D01B68002BDFD0210053
:1075C0005048F3E7504B1B68002BD8D05B68002B6A
:1075D000D5D021004348E9E7FFF7EAF9CFE78088F3
:1075E0004A4B984203D04A4B984200D070E7464B32
:1075F0001B68002BC3D05B68002BC0D02100D5E7EF
:10760000153B012BBBD963E7FFF798FAB7E7FFF704
:107610007DFAB4E73F4B1B78042B07D100236A4661
:1076200013800179408800F0C5FCA8E7364B1B6841
:10763000002BA4D05B68002BA1D0010036489847EE
:107640009DE7012421420AD0294B1B68002B04D05E
:107650005B68002B01D000209847012043E78B078F
:107660000AD5264B1B68002B04D05B68002B01D089
:1076700020009847022036E70421280008400D42E8
:1076800000D131E7254E3388002B21D0013B9BB23E
:107690003380002B1AD1FFF7DBF800280AD0204BEB
:1076A0001C70164B1B68002B04D05B68002B01D0AC
:1076B00020009847FFF7C6F8694601F001FD6846CB
:1076C000FEF7FEFF1D20FEF753FF308004200AE77F
:1076D000024B187804F0C4F8F8E7C046385FFF1F83
:1076E000BD3DFF1F0E20000001200000091000001A
:1076F000305FFF1FFEDFFFFFAFDFFFFF345FFF1FC5
:107700000C2000000B200000185FFF1F0D20000060
:10771000132000000D5FFF1FFFFF00000A5FFF1F27
:10772000085FFF1F10B501F09BF910BD014B1860F9
:107730007047C046345FFF1F0B880020162B01D80E
:1077400017230420014A13807047C046E25EFF1FE2
:1077500000207047074A03001188814207D09188B2
:107760000020994202D1013080001018704700209B
:10777000FAE7C046405FFF1FF0B58F7806000D00A6
:10778000C5B01E2F15D1FFF7E5FF051E03D100245C
:10779000200045B0F0BD00223B003100C0780092CF
:1077A00000F0B2FB0400A81C00F0D2FBFF23EB703A
:1077B000EEE7264B062403931B78FF2BE8D0182F07
:1077C000E6D87B08224A013BDB0002929A58944695
:1077D000002ADDD0029AD3185B68002BD8D0087835
:1077E000002802D14B78012B02D10624122FCFD1D1
:1077F00007AFAB88697800976446AA68A047041E63
:10780000C6D1AB78029A5B08013BDB00D318390084
:1078100030005B689847041E0BD1AB78042BB6D0C0
:10782000039A310010782200009700F06DFB0400ED
:10783000AEE76A78002AABD1AA7805A93B8808711F
:1078400030000A704B80FEF747FBA0E7C03DFF1FEA
:10785000CCBD00111D4B37B5050098420BD0002957
:107860000AD1FFF777FF002805D11948FFF772FF0B
:10787000002800D0058037BD01291AD1FFF76AFF23
:10788000041EF8D001235B420380A378FF2BF2D0C3
:10789000FE2B07D00023E0781422009329001E332A
:1078A00000F032FBA01C00F053FB01235B4263801D
:1078B000E1E70229DFD1013901F0BEF80028DAD171
:1078C0002800FFF747FF041EDFD1D4E7FEFF0000CA
:1078D000FFFF0000022210B5074B52421A800748F2
:1078E00001325A809A80DA8000F07EFA044801F072
:1078F00025F8002010BDC046405FFF1F79770011BA
:10790000557800110388F7B50400002B02D1022539
:107910002800FEBD42680221137825485268FEF710
:10792000A5FD00282ED0234F01253A88002AEFD04C
:10793000802321885B0201259B1A9942E8DC0C20F8
:1079400004F02EF9061E31D03B8822889C46002385
:107950001800019561469DB2491989B2AA421BD807
:10796000002801D062443A8000233000082208C079
:10797000210003F09DFF104A1368002B13D100254E
:107980001660C5E76268022113780C485268FEF75A
:107990006DFD0028C7D1BAE760681D01401941811B
:1079A00001330198D6E71A001B68E6E71325AFE715
:1079B0003ABE0011BE3DFF1F3C5FFF1F38BE0011E5
:1079C000014B18707047C046C03DFF1F14230A00CA
:1079D00010B51A40194204D00122102101F048F8D4
:1079E00010BD4B06F9D4012088434000F8E710B5DC
:1079F00014008B0604D50122102101F039F810BDC6
:107A000008230A001A40194202D14BB2002B0FDAA8
:107A1000102101F02DF8002808D02300F2331B7844
:107A2000002BECD0F1342378012BE8D10020E6E7DD
:107A300003208907FAD4E2E7F0B51F00184B85B0A0
:107A40001C68019002910392002C27D1200005B000
:107A5000F0BDA5683301ED186B89019A934211D3EB
:107A6000029A93420ED8002F04D10A9B002B10D10A
:107A70002C00EBE73B002978039A6868FEF7F6FCD8
:107A80000028F2D10136B6B2A388B342E1D8246807
:107A9000DAE7A3680A9A5B891380E9E70026F3E72F
:107AA0003C5FFF1F37B50C000A88498801239142CB
:107AB00017D3002A15D0651D23792A0002210A4810
:107AC000FEF7D4FC102300280BD02379618820888E
:107AD00000242A000094FFF7AFFF0A23A04200D041
:107AE000230018003EBDC0463ABE001113B50A007F
:107AF00008884988012388420BD8002809D000242F
:107B0000137905320094FFF797FF0A23A04200D0B3
:107B10002300180016BD13B50A0008884988012300
:107B200088420BD8002809D000241379053200942C
:107B3000FFF782FF0A23A04200D02300180016BDE1
:107B4000F0B58BB003904A8808880E00012382426A
:107B500055D3002853D00023012704AC2370002202
:107B6000718813000092FFF767FF051E3ED0207852
:107B7000002835D12B78022B18D167706A898300D1
:107B80000130E31880005A8069680222201803F04F
:107B90008FFE23780133DBB22370042B19D93B000D
:107BA0006889013080B2002BD9D01FE002236370B6
:107BB000122358436A89231804305A8069681022B6
:107BC000201803F075FE23780133DBB22370002BFD
:107BD000E5D10C4A6B899B185A425341DBB2DFE76F
:107BE0006378012BE4D12B78022BC7D022780A23AB
:107BF000002A04D021000398FEF798F9002318000A
:107C00000BB0F0BD0100FFFF0F4BF0B5040018688A
:107C1000002816D083685D89A54207D88288AE18EF
:107C2000B44203DA12019A18934201D10068EFE7D7
:107C30001E005F891036A74204D1002900D00D80B4
:107C40001800F0BD3300EFE73C5FFF1F70B5050083
:107C50000C0008880021FFF7D7FF03000120002B4C
:107C600004D022002800197AFFF7C1FE70BDF7B5D5
:107C70000C00002501902300EE331B78AB4201D8A5
:107C800000200AE06B00E65A00213000E718FFF7F9
:107C9000BBFF002802D126800130FEBD017A019889
:107CA000FFF794FE002802D03B882380F5E70135DA
:107CB000EDB2E0E710B5040008880021FFF7A4FF4B
:107CC00003000120002B03D02000197AFFF77EFE6D
:107CD00010BD0000054B1B68002B01D1180004E00B
:107CE0009A6852898242F6D1988870473C5FFF1F9C
:107CF000F0B50E27002687B0039302ABFF183E8035
:107D000005001F4B40891400984207D02B780130A2
:107D100000976A6880B2FFF78FFE060002212B7879
:107D200018486A68FEF7A2FB00280FD06C89200073
:107D3000FFF7D0FF002802D0013C0419A4B2039B36
:107D4000002B00D01C80300007B0F0BD02212B7842
:107D50000D486A68FEF78AFB0028E7D102212B78DC
:107D60000A486A68FEF782FB002807D0002EDED0A2
:107D70003B88A342DBD17489013CDFE76C89DEE7F5
:107D8000FFFF00003ABE001138BE001136BE0011E0
:107D900010B50C00FFF7DEFC03000220002B0AD018
:107DA000002C00D023609B781720FE2B03D00138D5
:107DB000FF2B00D1002010BD73B50D0001A90400F8
:107DC0001600FFF7E5FF172805D0002E04D1290083
:107DD0002000FEF727F976BD01221021200000F0D7
:107DE00047FE0028F3D0F6E7014B18607047C04605
:107DF0004C5FFF1F37B56B469D1D0100040002223A
:107E0000280003F06DFD2B88B02B0ED12379122BA7
:107E100009D12300FA331B78012B06D10121608898
:107E200000F0E0F801E01B2BF8D037BD10B5054B92
:107E30000421187000F098F8FFF74CFDFEF770FB76
:107E400010BDC046505FFF1F0020F0B50BB20F0001
:107E500087B0834234DA274B187803F031FD051ED2
:107E60002BD00378A02B25D103AE3100FEF7E4F828
:107E7000041E0BD1B378DB0724D51F4B06341B68D7
:107E8000002B03D03100688898470400A8680028B8
:107E900001D003F0D5FB002C08D1184A039B1340F6
:107EA000174A934206D0B3781B2B03D00121688870
:107EB00000F098F8280003F033FC8020000278409E
:107EC00007B0F0BD0F4B1B68002B10D03100688845
:107ED0009847041EDAD07378002BD7D1B27801A965
:107EE0000A704B800C716888FDF7F6FFCEE7062418
:107EF000F1E7C046505FFF1F485FFF1F00FFFF0014
:107F0000000112004C5FFF1FF7B50190FC200D002F
:107F100017001E0003F06CFB04001320002C12D08D
:107F2000B02320002370089BF422677065802671BF
:107F30000830002B08D0190003F0BAFC210001988A
:107F400003F006FD0020FEBD089903F0D9FBF5E71C
:107F500010B5041E06D00078FD2803D803F0F0FD0C
:107F6000FF23237010BD00000A1F93B210B5040058
:107F70000220032B05D882400020024BD1529B18CF
:107F80009C7010BD705FFF1F0B8870B5043B040030
:107F90000D000220032B0BD80121200000F04CFD26
:107FA00003001420002B03D02900200000F0DEFB8A
:107FB00070BD000007B51300034A00920A000121BA
:107FC00000F02CFC0EBDC046F181001107B50192F6
:107FD00003220092024B0A00122100F049FC0EBD60
:107FE0006F82001107B56B4601AA11800449D88041
:107FF00008780633012802D1190003F0B9FB07BD48
:10800000515FFF1F0C4B10B518700023FF210B4A66
:108010001380138193819380094A538013705172A6
:1080200093819372D174D3821375517703F0F8FC66
:1080300000F0FCF910BDC046805FFF1F705FFF1F9E
:10804000525FFF1FF0B58DB06B46002003910C22EC
:108050009B5E834200DBB0E05D4B187803F030FCA0
:10806000051E00D1A4E00378902B00D09DE006AF60
:1080700001004688380000F013FA796804000029EE
:1080800000D19CE03B88052B6ED13B89032B1CD98A
:1080900005AC200000F0A2F86288172A61D839895F
:1080A000131D994231D17968237804310291D9079F
:1080B00038D5607800F08EF9071E06D000230371D2
:1080C0002378012B08D0132B23D0A868002800D1D7
:1080D00078E003F0B5FA75E06288029909A800F02B
:1080E000A6F80290380000F08BF909AA2378387AB4
:1080F0000192002231000092029A00F012F9380039
:1081000000F064F9029B002BDFD0300000F080F912
:10811000DBE70378032BD8D16288029909A800F025
:10812000D6F8DEE7122B13D1029909A800F0B5F8B2
:10813000021EEAD127498B88002BC6D0887909A96D
:108140002378019161780091310000F0EAF8BCE7F2
:10815000002302AA93833000617809AAFFF72AFF5F
:10816000B3E71D4B0993F6E7042B02D09A1F012AAF
:10817000ABD8184A043B9B00995A0029A5D0D218C5
:10818000907831003A0000F0AEF800289DD13B888D
:10819000042B03D001213000FFF724FF012C04D170
:1081A000A868002801D003F04BFA280003F0B8FAC1
:1081B0008020039B0002434018000DB0F0BD012851
:1081C00000D182E701213000FFF70CFFEDE7C04648
:1081D000805FFF1F705FFF1F010017000B780370A7
:1081E0004B784370CB788A781B02134343807047E7
:1081F0000A88030002700A88120A42700A88012A5B
:1082000006D14A8882704A88120AC27004207047D8
:1082100002208242FBD14A8804309A704A88120AAE
:10822000DA708A881A718A88120A5A71EFE710B5D3
:108230000400012082420CD94B780A781B021343B8
:108240002380834206D1CB788A781B021343638054
:10825000002010BD022BFBD1CB788A781B02134380
:1082600063804B790A791B021343A380F0E70B88E4
:1082700003700B881B0A43704B8883704B881B0A62
:10828000C3708B8803718B881B0A4371CB88837101
:10829000CB881B0AC3710820704703000120082AFD
:1082A00014D14A780878120202431A80CA78887872
:1082B000120202435A804A790879120202439A80D4
:1082C000CA798879120202430020DA80704710B51B
:1082D00004000120022A05D100204B780A781B02F5
:1082E0001343238010BDF8B5060010200F001500C1
:1082F00003F07EF904000120002C0ED0A0230C22F4
:10830000290023806780201D002D07D003F0D0FABC
:108310002100300003F01CFB0020F8BD03F0F0F951
:10832000F6E7F7B51E00009008AB142017001D7883
:10833000019103F05DF9041E12D0A2230370019B8A
:1083400047704380099B057146710C220830002B51
:1083500007D0190003F0ACFA2100009803F0F8FAF6
:10836000F7BD099903F0CCF9F6E737B5041E0FD035
:108370004388002B0CD00025C1881323007A1722D4
:1083800001950095FFF7CDFFFF236580637225708F
:1083900037BD000010B50C4904004A88002A09D0F6
:1083A0008B89002B05D00020CB8A0222834201D08A
:1083B00010BD012213000A20434300204032C8545C
:1083C000C81842800472F3E7525FFF1F0023438006
:1083D00003707047094B00211A0010B55C88002C0F
:1083E00006D01C79844203D10A234B43D01810BD18
:1083F00001310A330329F1D10020F8E7525FFF1F52
:1084000010B50400407A03F09BFBFF23637210BD9C
:108410007047043010B580B203F0DAFA002803D0B8
:108420000421494203F00CFA10BD000070B500258C
:10843000104CA0682580A581A580A84202D003F039
:10844000FFF8A56000250C4C0C4B606D1D802300CF
:1084500058331D70A84202D003F0F2F8656500257C
:108460006068002801D003F0EBF8013508340A2DCC
:10847000F6D170BD1860FF1FBC5FFF1F0C60FF1FAF
:1084800070B5041E09D1054D2880A881A880A86870
:10849000002802D003F0D4F8AC6070BD1860FF1F54
:1084A000F0B54B8885B00193002343600A7905003D
:1084B0000F00022A00D07BE0CA88032A17D98B68F4
:1084C0005E7819783602DC78D8790E4399781B7A71
:1084D00024021B020C43034353495BBA0B80331D38
:1084E00093421ED1042C04D0631F022B0ED901200D
:1084F00015E0019A4D4B1201D35A002B06D001987A
:10850000FFF7BEFF4A4A1369013313610421B868BB
:108510002E812C80494203F093F96860002005B059
:10852000F0BD434D042C06D0631F022B0FD9EB681E
:108530000133EB60DBE7019A3C4B1201D35A002B6D
:1085400005D00198FFF79CFF2B6901332B61374B56
:1085500030000293019B029A1B01019300230199B1
:108560008C468B52130063449C8003939E81FFF7DB
:1085700050FF039B041E986016D00421B86849423E
:1085800003F05EF9FA880100043A200003F090F944
:108590000199029AFB888A5A043B9B18029A8B52D3
:1085A0002B6801332B60A2E7AB690133AB619EE717
:1085B0001E4B0293019B1E01029BF35A002B2DD0F0
:1085C00002998C19A068002828D0012A26D1FA889F
:1085D0009B189BB27352A189994217D39B1AC0185A
:1085E000B96803F065F9029BA289F35A934200D05F
:1085F0007DE700222B81A3882B80A3686B60029B00
:10860000F2520B4A53680133536070E7084A93688B
:10861000013393600198FFF733FF68E7044A536919
:1086200001335361F6E7C046825FFF1F1860FF1FEA
:10863000885FFF1F70B5051E15D10B4C0B4B1880C2
:10864000230058331870606D002802D002F0F8FF44
:108650006565250050356068002801D002F0F0FF04
:108660000834AC42F7D170BDBC5FFF1F0C60FF1F28
:10867000F0B51700A12285B0920001934243394B17
:1086800006001B680C009B18D933FF331D78FDF7DB
:1086900041FF0430854204DD3000FDF73BFF04302C
:1086A000C5B2BD4207D33A0000213000019B03F060
:1086B00057F805B0F0BD2900380002F081FF230013
:1086C000C6B250331E700393019B290063653800C6
:1086D00003F0BEF9CBB20293002B02D0039B01360C
:1086E0001E7000262300503303931B78B34204D836
:1086F000606D002831D10020DBE7029A2800002AB3
:1087000004D0013B1000B34200D02800F700E71965
:10871000387003F02DFA786000280ED03A7801996D
:1087200003F0C6F8019A3B780136D3180E4A01933C
:10873000D369F6B20133D361D4E7039B1870606547
:10874000A74205D1084A1320D36A0133D362B0E7A8
:10875000606802F075FF0834F2E702F071FF002351
:108760006365C8E73409FF1F885FFF1FF7B50D0079
:1087700007000421686803F063F82B890400037084
:108780002B891B0A43702B8883702B881B0AC370AC
:108790002E8902250436F6B2F42E15D81B4B9F42C3
:1087A00014D10C2002F024FF1135011E0CD09023AF
:1087B00003708E3B0371043B4380154B8460C6807D
:1087C000187803F0C5F800252800FEBD5C237B4324
:1087D000104AD3180093583301931B78002B0FD104
:1087E0000300320038000099FFF742FF019B0500AB
:1087F0001B78002BE8D13800009902F031FFE3E745
:10880000054A0725536A01335362DDE7FEFF000086
:10881000805FFF1FBC5FFF1F885FFF1FF0B587B041
:10882000009017200F0016000193FFF7F2FD1325AB
:10883000041E19D00C98031E02D00199201D9847E0
:10884000030AE370052302AAA07004309081277008
:108850000098667003A993800494FFF787FF051EB4
:1088600002D0200002F0ECFE280007B0F0BD0000AE
:10887000F0B587B01F000CAB1B7803910593012165
:108880000DAB06001C78049200F0D6F814250028E1
:1088900021D02000FFF77EFD0135041E1BD01149B9
:1088A000059B0A7803700132D2B2131EC68001D133
:1088B00001231A000B7022713000049B039900976A
:1088C000FFF7ACFF051E09D1230021000648074A27
:1088D000093303F035F8280007B0F0BD00236380AA
:1088E0002370F8E7845FFF1F6B8300113075000071
:1088F000F8B505000E00064C064F2368002B02D089
:108900003100280098470434BC42F6D1F8BDC04677
:108910002860FF1F3C60FF1F0123064A5B42538013
:10892000002313715362044A136053609360D36051
:10893000136170473C60FF1F2860FF1F0200002387
:1089400010B506499C000859002801D1625010BD9D
:108950000133052BF6D11320F9E7C0462860FF1F2D
:10896000034A5388181A4342584140421040704706
:108970003C60FF1FF0B585B002930AAB1F780CABCB
:108980001B88009008000E0001920393FFF7E8FF98
:1089900005001120002D1BD10E48FFF7E1FF040058
:1089A0001520002C14D006220B99A771E01D02F0AF
:1089B0007FFF019B30002371029B29006371009BA4
:1089C00066802370039B6562E381FFF791FF2800B7
:1089D00005B0F0BDFFFF000010B5FFF7C1FF0400B8
:1089E0000220002C12D060880121FFF781FF606A0D
:1089F000002801D002F0D4FE28220021200002F03D
:108A00007FFE012300205B426380207110BD0000C7
:108A100030B5074A074C5588010013780020A5425D
:108A200004D05B1A59424B415842104030BDC046F9
:108A30003C60FF1FFFFF0000084A10B501230C0037
:108A4000904208D0FFF78CFF031E04D00379234027
:108A50005A1E9341DBB2180010BDC046FEFF000055
:108A6000024B1879431E9841C0B270473C60FF1F0B
:108A700070B504000D001600FFF772FF002804D146
:108A80000D4B9C4200D0143070BD416A0379052023
:108A9000002907D012221A40102A02D10520002EE8
:108AA000F2D10F20DB06EFD5897E0C20A942894147
:108AB000494249420840E7E7FEFF0000030010B5C5
:108AC000002800D110BD0348034A41889142F9D0E3
:108AD0009847F7E73C60FF1FFFFF0000002330B519
:108AE000C45CCD5C6C40D4540133102BF8D130BD44
:108AF0000F23002210B5C45C64002243CA54C25C38
:108B0000D209013BF7D210BD0200010010B520329E
:108B1000103102F0D5FD10BDF0B58BB003901020E0
:108B200005931700049103F03BF80090102003F028
:108B300037F8009B13240190002B05D000280CD19E
:108B40001324009802F02CFE019B002B02D0180089
:108B500002F026FE20000BB0F0BD102003F020F83C
:108B60000600102003F01CF813240500002E00D18D
:108B7000AEE0002819D01022002102F0C1FD320021
:108B80002900039802F09CFD041E0ED133787F2B40
:108B900051D830000099FFF7ABFF009B1B787F2B6B
:108BA00053D801990098FFF7A3FF300002F0F8FDB9
:108BB000002D02D0280002F0F3FD002CC1D11020BE
:108BC00002F0EEFF0600102002F0EAFF0290002EF5
:108BD0007CD0002878D03A000F32230001251211F2
:108BE00005D00F333B4015B25A4253411BB26A1EA7
:108BF0001201002B33D0049BD2B298180099029A2C
:108C0000FFF76CFF013D10220021300002F078FDDB
:108C1000ADB2049F2D017D19AF4242D0002C33D05C
:108C2000300002F0BDFD029B002B00D189E7180047
:108C300002F0B6FD85E729003000FFF759FF280054
:108C40002549009AFFF74AFFA7E729000098FFF798
:108C50004FFF28002049019AFFF740FFA5E70F21A9
:108C60000F4004998A18D9B28F4208D9D15C06A85E
:108C700019540133102BF6D1029A0199C0E7791AE1
:108C800048424141C901F2E73900300006AAFFF726
:108C900025FF3200039806A902F012FD10370400E8
:108CA000BAE7002CBCD13000029906AAFFF716FFE4
:108CB000320006A9039802F003FD082204003100E7
:108CC000059802F0F5FDABE71324A9E71324AAE702
:108CD000002800D06EE733E740BE0011F0B58BB03E
:108CE0000F0016000225009000283FD0002A3DD03A
:108CF0000B1DDBB21800029302F052FF1135041E67
:108D000034D0FDF747FD05003A000099201D02F020
:108D1000EFFCEBB20393E3702B0CDBB22F0A009352
:108D20006370FFB22B0E2370A7700193FDF72CFD2B
:108D30001022010006A802F0DBFC2100029A04AB1D
:108D400006A8FFF7E9FE051E0DD1039B082233702C
:108D5000009B04A9B370019B7770F370301D02F083
:108D6000C7FCFDF71DFD200002F01AFD28000BB026
:108D7000F0BDF0B58FB00D00149E039004920593E2
:108D8000002A03D1022420000FB0F0BD002EF9D03C
:108D90000398FFF7E5FD1424071EF4D072783378AA
:108DA00012021A43B3781B041343F27812061A43D3
:108DB000036A0192934201D30133E3D1002D03D022
:108DC0003B7901249B07DED50822002106A802F08A
:108DD00097FC059B13240433DBB21800029302F0C6
:108DE000DFFE051ECFD0059A0499043002F080FC06
:108DF00004223100280002F07BFC390010221031DF
:108E00000AA802F075FC2900029A06AB0AA8FFF72F
:108E100083FE041E0FD1082206A908A802F068FCF0
:108E20000822311D08A802F0FBFB012807D1019997
:108E30000398FDF7C9FC280002F0B2FCA3E7012467
:108E4000F9E7000070B51C4C05002368181E10D00F
:108E5000002D14D11A78002A0CD1981C083202F087
:108E600027FD02F0B5FB0135002808D123681D70ED
:108E7000012070BD0A331800082202F019FD236892
:108E8000002BF5D0122002F0B3FB061E0DD0C1233B
:108E900021680370457002311022023002F008FD93
:108EA00023683100587802F053FD206802F078FC06
:108EB00000232360DCE7C0466460FF1FF8B50400B0
:108EC0002020FDF755FB0D4EA700BB590500002BD8
:108ED0000DD000280BD0D878FF2809D108492A00E6
:108EE0000C55F35907480333611802F029FDF8BD0A
:108EF000290002F005FE0028F0D1F8E78060FF1F8E
:108F00006860FF1F15A1001170B5064D84006359FC
:108F1000002B05D0D87802F013FEFF226359DA70D7
:108F200070BDC0468060FF1F70B506008CB00C009D
:108F3000150000213022684602F0E2FB31001022C9
:108F4000684602F0D5FB1D2021000322684402F090
:108F5000CFFB6846FFF7D8FD2D210400032228002F
:108F6000694402F0C5FB20000CB070BDF0B50700ED
:108F7000160097B001931CAB1D7830221EAB0091F8
:108F80000AA800211C7802F0BBFB102239000AA8B5
:108F900002F0AEFB1022002102A802F0B1FB072272
:108FA000310002A802F0A4FB072202AB9818631E4E
:108FB0009C41019902F09CFB02AB9C732B005A1E52
:108FC000934102AAD3730021102206A802F098FB55
:108FD00006221D9907A802F08BFB1A2002ABC018CD
:108FE00006221F9902F084FB102200990EA802F0BD
:108FF0007FFB102202AB0EA908781C78013A604072
:10900000D2B2087001330131002AF5D10AA8FFF766
:109010007BFD102212A904000EA802F049FC1022C8
:1090200006AB0EA908781D78013A6840D2B20870E4
:1090300001330131002AF5D10AA8FFF765FD044389
:1090400010222098E4B212A902F052FB200017B0BF
:10905000F0BD70B50E0014008CB0010010226846FF
:109060001D0002F045FB3100082204A802F040FB7D
:109070002100082206A802F03BFB6846FFF744FDEA
:1090800004001022280008A902F032FB20000CB0D6
:1090900070BDF8B506000D0000243719AC4200D3AE
:1090A000F8BD02F09DFB030A3B70631CDBB2013785
:1090B0009D4203D90234F054E4B2EEE71C00EDE720
:1090C00073B506000C000225002819D0002917D01E
:1090D000032101A8FFF7DDFF6B469A793F231A4071
:1090E000013313436A463000937101A92200FFF750
:1090F0001BFF051E04D10322E01C01A902F0D8FBCE
:10910000280076BD03785807DA08C00FD200800027
:109110009B0710439B0F1843C0B2704707230B40B7
:10912000C908C9000B4303707047000070B5040004
:10913000FFF7EAFE134DA4006359002B21D0186AF3
:10914000002801D002F02CFB2B59986E002801D08A
:1091500002F026FB2B59D86E002801D002F020FB2C
:109160002B59186F002801D002F01AFB2B59586FA9
:10917000002801D002F014FB285902F011FB002353
:109180002B5170BD8060FF1F0E4B8000C35870B51F
:109190000C00002B0FD09D68002D0CD02B78201DCB
:1091A0000B706B784B70A97CFFF7B8FF2B7E237296
:1091B0006B69E36070BD10220021200002F0A0FA6C
:1091C000F8E7C0468060FF1F014B18607047C0463B
:1091D0007C60FF1F074A03008000825810B5002AF8
:1091E00006D0D088984203D1012901D1FFF79EFF14
:1091F00010BDC0468060FF1FF0B5264E95B08700B9
:109200000B93BB590500099112200A92002B31D013
:10921000D888FFF7A5FB04001420002C2AD02800D2
:1092200010A9FFF7B1FFBB591E781D6A002E23D08D
:109230000895FDF7EFFA07000020FDF7F1FA079017
:10924000A379E61D069310AD0CA9089800F0E2FA88
:109250000EA9280000F0D7FA0B9B0A990493069BED
:1092600009980293079B0396019300970EAB0CAAF3
:10927000FFF77CFE15B0F0BDFDF7CCFA069030008C
:10928000FDF7CEFAE31DA779079310AB060008930C
:10929000DAE7C0468060FF1F30B50C4C85002A59C4
:1092A000030085B00120002A0ED018006946FFF7A0
:1092B0006BFF2B591A78D888054B002A00D1054B33
:1092C0006A46072100F0D9FB05B030BD8060FF1F62
:1092D000079800111598001130B5094C85002959DF
:1092E00085B010226846253102F0E2FA2A59112190
:1092F000044BD0886A4600F0C0FB05B030BDC046C4
:109300008060FF1FB198001130B5094C85002959C4
:1093100085B010226846353102F0CAFA2A59112167
:10932000044BD0886A4600F0A8FB05B030BDC046AB
:109330008060FF1FEF980011F7B54D4F8600102099
:10934000F4590D0002F02CFCF3592062186A132224
:1093500000286CD0033A29009C6802F0A9FAF3595E
:109360001A780192002A58D11E6A227D317B9446D8
:1093700051400122019F114201D167461740217DD2
:10938000914339432175377B4F40BC4660460027E7
:10939000800701D44F081740012102208F40227D11
:1093A00082433A432275377B5740BC4660460027CC
:1093B000400701D497080F400420227DBF0082435C
:1093C0003A432275627D002794466046727B424094
:1093D0000A4201D167460F400121627D8A433A4328
:1093E0006275777B5740BC4660460027800701D4F2
:1093F00057080F400220627D7F0082431743677544
:10940000767B00227E40760701D4BA080A40042603
:10941000617D9200B1430A4362756A78002A08D0E0
:109420006278002A05D005220533DA770022100081
:10943000FEBD04222979114205D1A17C114202D13D
:109440000533033AF1E7019A21782C78002A02D1FA
:109450000A002100140018220429E8D8042CE6D8B8
:1094600005206043034A05331218525CDDE7C0460D
:109470008060FF1F50BE001110B50A001121024B81
:1094800000F0FBFA10BDC0464B9900110B0030B53F
:1094900087B001AD2B806B4604001100981D082297
:1094A00002F006FA2A000B212000024B00F0E5FA38
:1094B00007B030BD7399001110B50A001121024B9D
:1094C00000F0DBFA10BDC046C799001113B50B00C0
:1094D00011006A4613706B4604000622581C02F005
:1094E000E7F96A4608212000014B00F0C6FA13BDD7
:1094F000E799001110B50A001121024B00F0BDFAE6
:1095000010BDC046379A00117FB505000B4BAA006D
:10951000D4580800002C0FD0666F237FE288217892
:109520000396266F0296E66E0196A46E0094FDF7F0
:1095300009FC2800FFF7FAFD7FBDC0468060FF1FD1
:1095400010B51721FFF7E0FF10BD000070B50A004D
:109550000D00064B0221040000F08FFA0600297866
:109560002000FFF7D1FF300070BDC04617990011F1
:1095700070B586B000236A461370836804001D78B6
:10958000681E0A2859D801A902F02AF806063337BE
:109590003B3F43474B4F5300180000F042F906236E
:1095A00012284BD000281BD16088FFF7D9F9082377
:1095B000002813D04279002A47D1264B1A78072376
:1095C00012070BD5244B1A680723002A06D0166809
:1095D000002E03D0290001AAB04703006A46137089
:1095E0006B461B786088002B2AD1FFF767FC06B01A
:1095F00070BD180000F06CF9D4E7180000F087F98E
:10960000D0E7180000F093F9CCE7180000F0ADF9AE
:10961000C8E7180000F0C3F9C4E7180000F0F6F935
:10962000C0E7180000F0F6F9BCE7180000F013FAE4
:10963000B8E7180000F013FAB4E707236A4613707E
:1096400069466088FFF782FFD1E70523012AC5D16B
:10965000024BB8E70D5FFF1F7860FF1F7C60FF1FA4
:10966000F8B52C4F8600F35904000D00002B40D0B4
:10967000DA8882423DD15A78062A33D11A78002AF4
:109680002ED0012099681A6A097D014206D0157B07
:10969000054203D007225A700120F8BD0220014282
:1096A00004D0157B054201D00922F4E704200142D1
:1096B00004D0127B024201D00B22ECE7164B1B6850
:1096C000002BE9D05B68002BE6D020009847BB59FF
:1096D00000215B78122BDFD12000FFF715FFDBE7BD
:1096E0000E4BECE7112A04D1002900D032252900C5
:1096F000F2E7002D08D12000FFF732F9002803D04F
:10970000102302791343037121002800FDF798FA12
:10971000C2E7C0468060FF1F7860FF1F7C60FF1FAC
:1097200070B50E4E8500AB590400002B13D01B788A
:10973000002B11D10A4B1B68002B04D05B68002B57
:1097400001D02000984773595B78122B03D1002178
:109750002000FFF7D9FE70BD024BECE78060FF1FD1
:109760007C60FF1F7860FF1F094B8000C3581020EA
:10977000002B0CD01A6A002A09D09B68002B06D057
:10978000127A1B7E101C9A4200D9181CC0B2704776
:109790008060FF1F70B503000D0014000220002A36
:1097A00030D000292ED013700B78081D53704B78E1
:1097B0009370FFF7A7FCE070012002212B7A237140
:1097C0006B7B034063716A7B0A401343042263711D
:1097D0006E7B1640334363716E7BF608F6003343AD
:1097E00063712B7B0340A371287B014000200B4356
:1097F000A371297B0A401343A3712A7BD208D200AC
:109800001343A37170BD10B50A0001000120FFF7DA
:10981000C1FF10BD10B50A0001000220FFF7BAFF1A
:1098200010BD70B506000C000220002E30D00029BB
:109830002ED07378201D0B70B3784B70F178FFF742
:109840006DFC01223579257271794B1008001340A7
:10985000934010400343881010408000C908034320
:10986000C9000B436373B1794B1008001340934058
:1098700010400343881002409200C9081343C900F6
:109880000B4321202373FCF773FE854201D2122083
:1098900070BD2220257AFCF76BFE8542F7D823782D
:1098A0001820042BF4D86378012BF1D80020EFE7BF
:1098B000030010B50220002909D0002B07D0032295
:1098C000481C0A7019000D3201F0F2FF002010BD93
:1098D00003000222080010B5002B06D0002904D096
:1098E0000E32591C01F0E4FF0022100010BD0300ED
:1098F00010B50220002909D0002B07D00422481CF3
:109900000A7019000C3201F0D3FF002010BD10B511
:10991000FFF7DEFF10BD03000220002906D0002B58
:1099200004D0052200200A701B784B70704703009A
:109930000220002B08D0002906D05B7800200B7095
:10994000013B082B00D918307047030010B50220E6
:10995000002909D0002B07D00622481C0A701900E4
:109960000A3201F0A5FF002010BD10B5FFF7B0FFCF
:1099700010BD02000B00022010B500290ED0002AF5
:109980000CD007211970118859701188090A997033
:1099900011180822D81C01F08BFF002010BD030015
:1099A0000A00022010B5002B0CD000290AD09978AB
:1099B0005878090201431180901CD91C082201F03B
:1099C00077FF002010BD030010B50220002909D048
:1099D000002B07D00822481C0A701900921801F0C9
:1099E00067FF002010BD02000B00022010B5002907
:1099F0000BD0002A09D00921197011781818597054
:109A0000511C062201F054FF002010BD10B5FFF7D5
:109A10005FFF10BD02000B00022010B5002A09D024
:109A2000002907D05178197011180622581C01F02E
:109A30003FFF002010BD030010B50220002909D00F
:109A4000002B07D00A22481C0A701900063201F0C8
:109A50002FFF002010BD10B5FFF73AFF10BD020028
:109A60000B00022010B5002A06D0002904D01800EF
:109A70005178FFF753FB002010BDF0B585B01700FB
:109A80001E006A4606230500080091819380FEF7B8
:109A9000C0FC1324011E02900CD03800B047041EF5
:109AA00005D1280001A9FEF76FFA041E02D0029822
:109AB00001F0C6FD2800FFF701FA200005B0F0BD57
:109AC000F0B504008BB0019115000021102202A80E
:109AD00001F016FE334EA700B85900283CD0C388C9
:109AE000A34239D10378002B36D14278062A18D107
:109AF00002000100553235310C3006ABFFF7A9FAF0
:109B0000002829D12000FFF72FFE020006A902A895
:109B100001F0CEFE200002A901F07AFE01200BB078
:109B2000F0BD816E002917D00B8A112A28D19D42E1
:109B30000ED101981231093A01F072FD012807D1C6
:109B4000BB5920009D6EFFF70FFE29000200DEE7E3
:109B500032212000FFF7D8FC2000FEF701FF061E8F
:109B60001BD0416A002918D00B8AAB4215D10822BC
:109B70000198123101F054FD01280ED1716A0AE0FA
:109B80009D42E9D108220198123101F049FD0128D6
:109B9000E2D1BB59996E8A7EB9E7200001F0A8FE98
:109BA000BCE7C0468060FF1FF0B56B4D87007E5953
:109BB00085B0337802900393002B00D087E0B36820
:109BC000346A01937078062817D101221B7D134255
:109BD00002D0217B114218D10222134202D0217BF4
:109BE000114251D10422134203D0237B134200D0EF
:109BF0008BE0019B5A7DEB5991E007380428F8D897
:109C000001F0EEFC032E42678300B36E002B03D1FC
:109C10001C2001F0C5FFB066EB599C6E002C1CD0D7
:109C200010220021200001F06BFD0298FFF79CFD3F
:109C300001002000FFF72DFA01F0D2FD2082200064
:109C400008211230FFF725FA0298FFF78DFDA07664
:109C5000EB592100D888FFF70FFC0822EB591CE0D4
:109C6000B36E002B05D01A00198AF0881232FFF764
:109C70000DFC0222019B197DEB5911423DD0207B46
:109C800010423AD0073208E0F488FCF7DBFD01000F
:109C90002000FFF711FC0A22EB595A70029B9C002E
:109CA0002A595378073B042B11D8D088FEF758FE69
:109CB00000284ED0C3895A08D2182849029B02981E
:109CC000CB542B5941180433254801F039FE05B017
:109CD000F0BDFCF79FFD03000120834201D100206D
:109CE0000393EB59DE88FCF79BFD039902003000DB
:109CF000FFF7ECFB019AEB59117D042211420CD0C5
:109D0000217B114209D00B22C7E7F688FCF73CFD06
:109D100001003000FFF7EEFB6BE7019A527D012155
:109D20000A4204D0607B084201D00C22B5E7022130
:109D30000A4204D0607B084201D00E22ADE7042124
:109D40000A4204D0627B0A4201D01022A5E7122207
:109D5000A3E7FA225200B0E78060FF1F8460FF1F74
:109D60001FA1001110B5064B1A78042310001840EB
:109D70001A4200D00348FFF727FA002010BDC04662
:109D80000D5FFF1FC43DFF1F70B50400FFF7D4FA3D
:109D9000051E43D12000FFF77FFA234EA400A059EF
:109DA0008268937CDB0708D50321036A1B790B408B
:109DB000012B02D1017F0B430377431DD97F8B1EFB
:109DC000022B0DD8022900D00121C088FCF790FF9A
:109DD000042133591A7F59700A431A77280070BD3D
:109DE00001290CD102231022437000210C3001F014
:109DF00087FC305910213530FFF74BF9EEE7052984
:109E0000ECD10223D118437010220C3001F050FD28
:109E100004233259117F0B431377EAE708251828EA
:109E2000DCD1053DDAE7C0468060FF1FF0B58BB09E
:109E3000059143887E4F9E00F45915000493002C31
:109E400015D1012902D000200BB0F0BD101D5778AC
:109E50001678FFF757F9EB68320002932B7A0499D2
:109E6000019300903B002000FCF70CFFEBE7E38838
:109E7000049A934201D00820E6E72378012B00D111
:109E8000D4E0059B581E092800D9CFE001F0A8FBBB
:109E900005CE0A29CC506C859AB229000498FFF7A8
:109EA00073FFD1E7200029001022453001F000FDAA
:109EB000B9594B78042B02D1013B4B70C3E70B001F
:109EC0000A00253335320C310498FFF795F90498D0
:109ED000FFF702FA0522431E9841BB59C0005A7091
:109EE000B2E7200029001022553001F0E1FC049B6C
:109EF0004F4C9D00295904980A0006AB55320C318D
:109F0000FFF77AF929591022453106A801F088FB9C
:109F1000012808D10498FFF7F7F90590002804D12B
:109F200006222B595A7005988EE708230593FAE705
:109F300063780C2B7AD1E36E002B03D11C2001F047
:109F40002FFEE066BB59D86E00286FD01022290082
:109F500001F0AEFCBB590498DC6EFFF705FC0D2246
:109F6000A076BB595A706EE7E06E00285ED0637829
:109F70000D2B5BD12B8808220382A91C123001F023
:109F800097FCBB599A68517D0222114226D0186A6B
:109F9000407B104222D00C32E4E763780E2B45D18F
:109FA000236F002B03D1162001F0FAFD2067BB5967
:109FB000186F002803D01022290001F079FC0F222D
:109FC000BB59CFE763780F2B30D1206F0622691C75
:109FD000103001F06DFCBB599A68517D042211428A
:109FE00003D0196A497B1142D5D100210498FFF7AB
:109FF0008BFA28E7636F002B0DD0BB59586F0028F0
:10A00000F3D01022290001F053FC0122BB59524227
:10A010005B6F1A61E9E7142001F0C2FDBB5960676C
:10A020005B6F002BE9D126E72978DFE707200BE7F4
:10A030008060FF1F10B5064C207001F009FC06215E
:10A040002078FDF791FF0348FEF778FC10BDC0466D
:10A050009360FF1FD591001100200BB270B50D0069
:10A06000834216DA264B187801F02AFC041E0DD024
:10A070000378922B0ED0A02B37D0224B1878FF28D4
:10A080003AD0210001F064FC002835D18020000284
:10A09000684070BD43780E2B0BD03E2BEDD18378FA
:10A0A000052B12D0082BE8D181798088FFF7D8FAE8
:10A0B00008E0154B82889A42DFD183681878591CD2
:10A0C000FEF7C0FE002817D1D7E7104B1B785B07BF
:10A0D00012D50F4B1B68002B0ED09B68002B0BD0AA
:10A0E000C289811D80889847ECE7FFF741FAA06894
:10A0F000002801D001F0A4FA200001F011FBC5E70F
:10A100009360FF1FBD3DFF1F182000000D5FFF1F64
:10A110007C60FF1F10B50078FFF712FA10BD10B574
:10A120000078FFF7FDFA10BD0C234343084A10B531
:10A130009B185A68002A03D0012901D1904710BD0D
:10A140009B68002BFBD00029F9D19847F7E7C04660
:10A15000B060FF1F01238340094A10B5946B1C4374
:10A160009463506B98435063D46B2000984301294B
:10A1700001D120001843D063116B0B43136310BD52
:10A1800000800040F0B500240127154B85B0DA6B44
:10A19000144E03921A6C0192DA64019BE3403B4235
:10A1A00017D0039DE5403D400295E5B20299280095
:10A1B000FFF7BAFF316A736A002908D03900002B13
:10A1C00001D0029979402800FFF7C4FF01E0002B7D
:10A1D000F9D101340C36172CDFD105B0F0BDC046E3
:10A1E000008000409460FF1F064B01215A68C24066
:10A1F0000A4204D01B68C3401800084070471B6D1A
:10A20000F9E7C046008000400122064B8240002949
:10A2100003D0D9680A43DA607047D9689143D9609E
:10A22000FAE7C0460038004030B5032444430F4BE2
:10A23000E25C1B199C785D7801232D1B0135AB4036
:10A24000013BA340A140DB430C00122807D808497A
:10A2500092005218116819402143116030BD054A1F
:10A2600011680B4023431360F8E7C04697BE001106
:10A2700008F0004014F00040C21F70B5D4B20623AD
:10A28000092C0BD80125084C9540002908D0002145
:10A29000FFF7CAFF23682B4323600023180070BD1B
:10A2A0002368AB43F8E7C04600380040214BF0B5C7
:10A2B0001B185B78022B21D1032444431E4A1F4EF6
:10A2C000A35C12199478012215008540B76B013CFC
:10A2D000E4B23D43A240B563194C122815D89B0047
:10A2E00000290CD117495B1899680A439A60012329
:10A2F000205C154A834011680B431360F0BD11497F
:10A300005B18996891439960F1E70E4B00290DD1D4
:10A3100059690A435A61225C1328E8D00123203A84
:10A3200093400A49086803430B60E7E75969914382
:10A330005961F0E79460FF1F97BE00110080004054
:10A34000DCBE001100F00040A0F00040A4F000408E
:10A35000F8B500241B4E1C4D1C4B1B5D012B1FD15F
:10A36000194A9269E2401A420BD00122B256934038
:10A370002200143AD2B2022A09D815494A69134375
:10A380004B61013402360C35172CE5D1F8BD0022A3
:10A39000B2560F499200521891680B439360F0E750
:10A3A000022BEED1E7B23800FFF71EFF0123584021
:10A3B000C1B23800FFF77AFF3800FFF715FF687762
:10A3C000DFE7C04669BE00119460FF1F9560FF1F64
:10A3D00000F00040012202388240054B002903D0E2
:10A3E00059690A435A617047596991435961FAE7BB
:10A3F00000380040F8B50E0001210F008740114AD7
:10A400000400D368FD43BB43D360831E8B4201D855
:10A41000FFF7E0FF00212000FFF72EFF0A4A0B4B59
:10A420005168012E05D139431B1951605E7000201F
:10A43000F8BD2940516002221C1962709A691540CA
:10A440009D61F4E700380040008000409460FF1FE9
:10A45000012210B58240074B002906D019680A4333
:10A460001A600121FFF7C6FF10BD196891431960FA
:10A47000F7E7C046008000400C2370B50025434339
:10A480000A4A29009B181D70094B04001B185D70B7
:10A49000FFF7B0FF0123A340064928000A681A43CA
:10A4A0000A6005490A689A430A6070BDB060FF1FE0
:10A4B0009460FF1F348000403080004070B504007D
:10A4C0000E00FF2813D003250540FFF7D5FF084AEB
:10A4D000A3089B009B183F22ED00AA40AE401968DC
:10A4E00020009143314319600121FFF78DFE70BDBB
:10A4F00018380040F8B50C244443134B0500E41809
:10A500006368002B03D1A3681220002B1AD002220B
:10A5100001270E4B00215B195A7028002770FFF7A6
:10A5200069FF63681E1E08D0A3683E00002B04D09C
:10A530002800FFF759FE4640F6B228003100FFF729
:10A5400009FE0020F8BDC046B060FF1F9460FF1FE9
:10A55000F7B5C420FF222B4B8000195800249143EB
:10A560003F3A0A431A508022274F5202274E1A6060
:10A57000274B1D5D002D21D0A31E012B03D80121E7
:10A58000E0B2FFF727FF012D18D11F4B9B69E34075
:10A590002B4213D0E3B218000193FFF725FE010010
:10A5A0000198FFF755FFE3B2143B022B1DD80121A0
:10A5B0007156184A8D405369AB4353613B7F002B62
:10A5C0000DD0E5B22800FFF795FF2800FFF70CFE3D
:10A5D0007B7F0100834202D02800FFF7A5FD0134F4
:10A5E0000C370236172CC3D1F7BD01210023715659
:10A5F000F3568D40074A9B009B189A68AA439A60BD
:10A60000DCE7C04600E100E09460FF1F69BE001176
:10A610009560FF1F00F0004070B50E0015000400AB
:10A62000FFF72AFF0C236343094A20009B189D6013
:10A630005E60FFF75FFFF021064B074A8900051EA9
:10A640005A5002D02000FFF717FF280070BDC04607
:10A65000B060FF1F0000FF1F85A1001170B5134DF2
:10A6600007202C78002C1FD19822210052002800AE
:10A6700001F05EF90123C420FF222B700C4B8000F7
:10A680001C635C630B4B1C605C600B4B1958914363
:10A690003F3A0A431A50802252021A600D20074A9C
:10A6A000074901F01DF8200070BDC0469460FF1FEF
:10A6B00000800040A0F0004000E100E051A5001142
:10A6C00051A3001170B51D0002240C2910D8094AAD
:10A6D000CA40D2070CD5FBF757FF041E08D1059AD4
:10A6E00004992800FBF76CFFFCF7DAFDFFF73AFB53
:10A6F000200070BD1210000030B50D7802232C0030
:10A700009C43184201D02B431C0008252300AB4377
:10A71000284201D02B00234320241D00A5432042C2
:10A7200001D01C4325002A230D70184204D0117853
:10A730001E3B0B43137030BD0028FCD10C21137855
:10A740008B43F7E7F8B51D0006AB1B88140007AA7A
:10A750000E000B201778002B27D10A78022A49D146
:10A760004A68507811780002244A08438018042867
:10A7700040D800F035FF03121D1B2300F06801F0E4
:10A7800077F8021CC0B2B84200D93A1CD2B22000FD
:10A79000F1682A8001F08CF806E00222F3681B8839
:10A7A0002A8023701B0A63700020F8BD0622EEE7A2
:10A7B00001232B80F3681B782370F5E7F368002BE7
:10A7C00016D008222A801A8822701A88120A62700B
:10A7D0005A88A2705A88120AE2709A8822719A885E
:10A7E000120A6271DA88A271DB881B0AE371DBE767
:10A7F0002B80D9E701202B80D7E7C04600D6FFFF8A
:10A80000F7B516000A781D0008AB1F880C0001235D
:10A81000022A18D14A685078117800022B4A08435E
:10A82000801803280FD800F0DBFE02254439E068C9
:10A8300001F01EF8C0B20723B84204D37B1901937C
:10A84000152B02DD0D231800FEBDE0682A00310043
:10A85000C01901F02DF86B4600209B88E268D054A7
:10A860001B4B1B68834203D01B68834200D0984770
:10A870000023E8E70B23002FE5D1022DE2D1737806
:10A8800032781B021343E2681380114B1B68002BC4
:10A89000EED01B68002BEBD00120E8E70B23002F44
:10A8A000D1D1062DCED12A003100E06801F000F8A8
:10A8B000DEE70B23002FC6D1012DC3D132787533CB
:10A8C000012AC0D8E3681A70D2E7C04600D6FFFF5D
:10A8D000A062FF1F70B50C001500072837D800F0E4
:10A8E0007FFE041436361B36242E182015290BD86B
:10A8F000184E16220021300000F002FF220029002D
:10A90000300000F0D5FF002070BD18200229FBD1D7
:10A910001288114B1A80F6E718200829F4D10A0092
:10A920000E48290000F0DCFFEDE718200129EBD1EB
:10A930000B4B10780B49DA69FFF7DEFEE3E71820CE
:10A940000129E1D1064B10780749DA6BF4E70220C0
:10A95000DAE7C0468862FF1F663EFF1F5C3EFF1FAE
:10A96000EC3DFF1F143EFF1F343EFF1F030010B5D8
:10A970000020DB0704D50721024A034800F08CF8C9
:10A9800010BDC046F4BE0011EC3DFF1F054A030098
:10A990001068002803D082889A4201D180687047ED
:10A9A0000068F6E79864FF1F0A88030008009A42CF
:10A9B00004D08A8804309A4200D0002070470000FA
:10A9C000F8B5F22200230D4F0D4E79680500424381
:10A9D0003370994200D07B600A4C0021200000F0C7
:10A9E0008FFE00231A007C60AB4202D1002033703E
:10A9F000F8BD01332280DBB2F234F5E79065FF1F2A
:10AA00008E65FF1F9C64FF1F73B56B4601900600A7
:10AA1000684615001980FCF775FF041E11D1002D42
:10AA20000FD07689002E11D00C2001F0B9F8002843
:10AA30000ED0084A0460136886808560002B02D11E
:10AA40001060200076BD1A001B68F7E70224F8E7C3
:10AA50001324F6E79864FF1F012100220A4B10B56A
:10AA600049420A4C198099809A719A70084B20705B
:10AA7000012019805A60FFF7A3FF2078FCF7A0FFA0
:10AA80000448FDF75BFF10BDA862FF1F9865FF1F1C
:10AA90009065FF1F45AB0011022310B5002802D0BE
:10AAA000FFF7B2FF0300180010BD0000030010B54F
:10AAB0000020DB0704D50421024A0348FFF7A4FF66
:10AAC00010BDC04608BF00116C3EFF1FF0B50E263A
:10AAD00087B003930CAB1F8802ABF6180500080083
:10AAE00031000292FDF790F804000120002C0FD0F5
:10AAF0003088FFF74BFF03000E20002B08D05E6864
:10AB0000002E05D021002800039B029A0097B04731
:10AB100007B0F0BD0A4B10B5984207D101220023BF
:10AB200052420A808B708A808B7110BDFFF73CFF08
:10AB30000028FAD001235B42038000238370F4E7EE
:10AB4000FFFF0000F8B5050001290AD1134E0024CB
:10AB50003388F227AB4219D028001149FFF7DAFFFA
:10AB600006E0022904D10139FDF766FF0028EDD087
:10AB7000F8BD3B0063437268D018D35A002B09D04C
:10AB80003A00002100F0BCFD0134E4B2054B1B7813
:10AB9000A342EED801235B423380DDE79065FF1FBF
:10ABA000A862FF1F8E65FF1F10B5FFF7FDFE0300B3
:10ABB0000020834200D0987810BD0000F0B589B025
:10ABC0001C000EAB80CB03901E8810AB1B78049248
:10ABD00002930B7A0D00DB0616D42B780593022B1B
:10ABE00024D00498FFF7D2FE002812D003689C46B8
:10ABF000002B0ED0029B2200019329003B006446EB
:10AC000003980096A04705E00498FFF7BFFE0028D0
:10AC100002D10E2009B0F0BD8368002BF9D00A22C2
:10AC20002900039898470028D7D0F3E76B68587835
:10AC30001A786B4B000210439842D2D8043B9842DA
:10AC400010D2684B984242D015D8674BC0180128E3
:10AC5000C7D80B20002EDDD1EB681A7859683A80EE
:10AC6000200028E0614BC018032800D979E000F0EB
:10AC7000B7FC846A789E5E4B9842B2D10B20002EBE
:10AC8000C8D101233B80EB6831001B7823706889B1
:10AC9000013080B2FCF7B8FF3A88031E0ED001786D
:10ACA00002328A183A80428962704289120AA2707E
:10ACB00059680278E01C00F0FBFD06E004323A809F
:10ACC00031000422601C00F01BFD0020A2E70B20D5
:10ACD000002E9FD1EB6807A91E8804233B80330A0E
:10ACE000300026706370FCF78FFF051E28D004AB80
:10ACF0009A890E2304A95B183E49C668FCF7F8FF41
:10AD000000280BD12B783C486A680599FBF7AEFB0D
:10AD1000002803D1012304AA5B42D3813278022A9E
:10AD200006D17168201D00F0C3FD3B8802333B80D3
:10AD30000E2304AA9B181B88A3701B0AE370C4E7A8
:10AD400004ABDE81F4E70B20002E00D062E7E96857
:10AD50000398FFF729FF02233B802070000A6070F0
:10AD6000B3E70B20002E00D054E70222EB681B88CB
:10AD70003A8023701B0A6370A7E7E86800F078FD4B
:10AD8000C2B203000720B24200D243E70DD00299BD
:10AD9000DBB27118994202DB921BD3B20293029B81
:10ADA000E9681A003B8089195AE70023F6E70B206F
:10ADB000002E00D02EE70722EB683A801A78227026
:10ADC0005A7862705A88A2705A88120AE2701A7908
:10ADD0002271DA886271DB881B0AA37175E7C046AD
:10ADE000042900000228000000D8FFFFFFD6FFFF63
:10ADF00003280000FFFF000038BE0011F0B58DB041
:10AE00006B460020089120229B5E83423DDAA64BD0
:10AE1000187800F055FD071E32D00378B02B2CD1E6
:10AE20000079023816281FD800F082FE17001E0095
:10AE30001E001E0031001E0096001E001D011E0097
:10AE400052011E0073011E00CD011E0050021E00A3
:10AE50001E001E008E021E00E302944B94491B88C4
:10AE600078880B80FBF742F83800FCF7C3FF914B62
:10AE70001B68002B01D038009847380000F050FCC8
:10AE80008020089B0002434018000DB0F0BDEE2268
:10AE90000021874800F034FC0BAA3B7B7989388974
:10AEA00000923A000D32FCF7C7FD0400804B1B787E
:10AEB000002C3FD146E0804B788805937F4B4100C2
:10AEC000CB5A0BAE073BDBB23288029300230193CF
:10AED0007B4B210006930093059BFFF76FFE744D9B
:10AEE000002810D1069B3A8A1B889A420BD1380061
:10AEF0000599123000F094FB002804D02B78628969
:10AF00009B00EB185A80162306A81B1832882000D5
:10AF10007989FCF7EDFE2B7804009A00AA18518875
:10AF20000029C3D00133DBB22B70002807D006A95B
:10AF3000C98A9180634A12889A42BCD802E00121F2
:10AF400049429180002B04D059497888FBF702F8D8
:10AF50008AE73E890A2479E000253E89574B06930B
:10AF60007B88069A5B009B5A033B9D4202DB002DC7
:10AF7000F0D05BE0162206A812183B7B798900927C
:10AF80003A0030000D32FCF757FD0590002858D0EC
:10AF90004689017A7888FCF719FD041E44D1464B96
:10AFA00078880793069B4100C95A454B0439C9B2BA
:10AFB00006AAD28A06930291019400930599079BF1
:10AFC000FFF7FCFD041E2FD1069B39491A88931CFC
:10AFD000002D26D14B807988384B4900CB5A511926
:10AFE000033B8B4220DD059B31485B8941190B7186
:10AFF000A91C0135C9B2EDB2059145191B0A2B7187
:10B00000059B2D490433181800F052FC2C4B059A6F
:10B010001B88D318DDB22C4B9E4205D00136B6B248
:10B020009CE749889942D6D0002D0CD0204C2800AE
:10B03000618800F06DFC207021007888FAF79AFF93
:10B0400012E7059CF0E7002C00D183E77B78142BF6
:10B0500000D109E716493B794E800B700C71788856
:10B06000FAF73AFF00E7162406ABE4182100388906
:10B07000FCF7CAFD011E00D1B7E1788822880F4C89
:10B0800045002C5B0A4D013CE4B2029400240F4BB6
:10B0900001940095FFF792FD041E00D014E12900F1
:10B0A0007888FAF777FFDFE69865FF1F5C3DFF1FA2
:10B0B000B062FF1FA462FF1FA463FF1FE05EFF1FBB
:10B0C0009464FF1F5A3DFF1FFFFF0000B262FF1F85
:10B0D000162406ABE41821003889FCF795FD011E03
:10B0E00000D182E178882288AE4C45002C5BAE4DC1
:10B0F000013CE4B202947C89AC4B01940095FFF7CB
:10B100005DFD041E00D0DFE029007888FAF74CFFCF
:10B11000AAE60025A44B1D803B00F6331B78A24A0B
:10B1200078880792AB4208D99E4B128806930699FD
:10B1300043005B5A013B9A4203DB0799FAF73EFF53
:10B1400092E616246B00FB18059306ABE418059BEA
:10B1500021001889FCF758FD011E03D1059B01242D
:10B160001E8973E77888924B2288069C09934300D6
:10B170001B5B904E013BDBB20293002300960193D0
:10B18000099BFFF71BFD041E02D0059B1E895DE78E
:10B190007B88069A5B009B5A079A1088328812189F
:10B1A000934202DC1B1A013B33807F4C0230328811
:10B1B0000999001900F07CFB2388328801359B181F
:10B1C0002380EDB2A8E70BAA3B7B798938890092EE
:10B1D0003A000D32FCF730FC00250590059B002B52
:10B1E00004D10A24002D00D16EE060E0059B788830
:10B1F000197AFCF7EBFB0100041E63D1694C6C4B20
:10B20000788806940993069B4400E45A694B063CEF
:10B21000E4B20BAE32880793029401910093059932
:10B22000099BFFF7CBFC041E4CD1079B5E491B8892
:10B230001A1D002D30D14A80059B5B4C5A89631939
:10B240001A716B1C9BB2E318120A1A71162306A816
:10B2500032881B1879890598FCF74AFDFF21AA1C42
:10B260002E1D03350B00059092B2B6B2ADB2002888
:10B2700003D006ABDB8AD9B21B0AA218651911717B
:10B280002B714C4D301D2A884949201800F010FBC5
:10B290002B88F618B5B2A1E74988914207D17A8880
:10B2A00006995200525AEB18053A9A42C4DC3E4CB9
:10B2B0002800618800F084F9207021007888FAF76E
:10B2C00087FED1E5002DF2D13E89BFE6162606ABFA
:10B2D000F61831003889FCF797FC3D000400FA3578
:10B2E00000282DD0037A9B060CD400227B89398953
:10B2F000788800923A000C32FFF7E8FB041E10D069
:10B300003E8915E03088FFF741FB00281AD083689A
:10B31000002B17D02100122278889847041EE4D011
:10B32000EEE72B78002B02D17888FAF761FE002631
:10B330002B78002B00D097E5002C00D194E585E612
:10B340000124DDE70E24DBE7162506ABED18290006
:10B350003889FCF759FC041E47D0037A9B0611D4A8
:10B36000154A7B881188994203D01448814207D13D
:10B370001380134BF2261D780023D9B2A94221D3A2
:10B380000924A1E72888FFF701FB00282FD0836854
:10B39000002B2CD02100122278889847041EDFD081
:10B3A00092E7C046E05EFF1FB062FF1FB262FF1F60
:10B3B000A463FF1F9464FF1F9065FF1FFFFF000041
:10B3C0008E65FF1F31005943546801336018615A7C
:10B3D0000029D2D13C0008342100F22200F068FAA2
:10B3E00021007888FAF70CFE3EE501246CE70E2474
:10B3F0006AE71D4B1A887B889A4231D07888FAF721
:10B4000009FE31E5F223059851684343CD18C95A26
:10B4100000291FD03B7A012B0BD16C88AB88788830
:10B42000AA1D0094FFF752FB041E02D000233B72BA
:10B430002E88F2220021280000F062F900232B80E0
:10B44000059B0133DBB20593084B05991B78064A2F
:10B450008B42D7D801235B421380002CCED0F5E578
:10B46000002634000596EFE79065FF1F8E65FF1FED
:10B4700070B504000E001500FFF796FA031E08D100
:10B4800031000548FFF790FA03001120002B02D08D
:10B490001C8000209D7070BDFFFF0000F8B50B4FB1
:10B4A00006003B780D001400FF2B0ED00A2000F0A0
:10B4B0009FF8011E09D0B123038000234680037149
:10B4C000C5800481387800F043FAF8BDAD3EFF1F17
:10B4D000F7B50F0008A90600088809A90B240988F8
:10B4E000002821D10234022B1ED1557813782D0269
:10B4F0001D432B008B4301937334002B14D1FB6845
:10B50000300019000093FFF74FFB019C85420BD0E0
:10B510002A0030000099FFF7ABFF041E04D12A0077
:10B5200030007989FFF7BAFF2000FEBDF0B50E7834
:10B5300085B003900AA805880120022E0DD14C6821
:10B540002778647824023C43054FBC4205D1039818
:10B55000DBB201960095FFF7BBFF05B0F0BDC0461A
:10B5600002290000034B10B51B68002B00D0984740
:10B57000FEE7C0469C65FF1F07B501A8FFF7F2FF75
:10B58000044A05480021121A00F0D2F9F8F732F9FE
:10B59000FEE7C046A065FF1FB03EFF1F0000000091
:10B5A00001B40248844601BC604700BFC9A900003D
:10B5B00001B40248844601BC604700BF2135FF1F2B
:10B5C00001B40248844601BC604700BF090E000078
:10B5D00001B40248844601BC604700BFD91B00008B
:10B5E00001B40248844601BC604700BF6136FF1FBA
:10B5F00001B40248844601BC604700BF1D4D0100F4
:10B6000001B40248844601BC604700BF55220000D7
:10B6100001B40248844601BC604700BF75A9000020
:10B6200001B40248844601BC604700BFCD4C010014
:10B6300001B40248844601BC604700BFDD660100DA
:10B6400001B40248844601BC604700BFD9490100EB
:10B6500001B40248844601BC604700BF3555000074
:10B6600001B40248844601BC604700BF7D18FF1F3B
:10B6700001B40248844601BC604700BF6D33FF1F20
:10B6800001B40248844601BC604700BFA534FF1FD7
:10B6900001B40248844601BC604700BF7932FF1FF5
:10B6A00001B40248844601BC604700BF4D36FF1F0D
:10B6B00001B40248844601BC604700BF2124000059
:10B6C00001B40248844601BC604700BFE548000061
:10B6D00001B40248844601BC604700BFF530FF1F3B
:10B6E00001B40248844601BC604700BF952BFF1F90
:10B6F00001B40248844601BC604700BF45510100C7
:10B7000001B40248844601BC604700BF154D0100EA
:10B7100001B40248844601BC604700BFF928FF1FFE
:10B7200001B40248844601BC604700BF434D01009C
:10B7300001B40248844601BC604700BFED4A0100E5
:10B7400001B40248844601BC604700BFB14E00000E
:10B7500001B40248844601BC604700BF4D35FF1F5D
:10B7600001B40248844601BC604700BF5118FF1F66
:10B7700001B40248844601BC604700BFE1170000E5
:10B7800001B40248844601BC604700BF691F000045
:10B7900001B40248844601BC604700BFC531FF1FA9
:10B7A00001B40248844601BC604700BF014C01005F
:10B7B00001B40248844601BC604700BFC51D0000BB
:10B7C00001B40248844601BC604700BF85520100B5
:10B7D00001B40248844601BC604700BF65710100A6
:10B7E00001B40248844601BC604700BF29510100F2
:10B7F00001B40248844601BC604700BF055E0000FA
:10B8000001B40248844601BC604700BF5D2DFF1FA4
:10B8100001B40248844601BC604700BF311B0000F0
:10B8200001B40248844601BC604700BF851F000088
:10B8300001B40248844601BC604700BFB933FF1F12
:10B8400001B40248844601BC604700BF554901006D
:10B8500001B40248844601BC604700BFC92600000D
:10B8600001B40248844601BC604700BFB3520100E6
:10B8700001B40248844601BC604700BFDD520100AC
:10B8800001B40248844601BC604700BF4D1F000060
:10B8900001B40248844601BC604700BF056A00004D
:10B8A00001B40248844601BC604700BFF52AFF1F6F
:10B8B00001B40248844601BC604700BFE94C010066
:10B8C00001B40248844601BC604700BFF54E010048
:10B8D00001B40248844601BC604700BFC521000096
:10B8E00001B40248844601BC604700BF810E0000DD
:10B8F00001B40248844601BC604700BF091B000038
:10B9000001B40248844601BC604700BF0D520100EB
:10B9100001B40248844601BC604700BF350E0000F8
:10B9200001B40248844601BC604700BFC530FF1F18
:10B9300001B40248844601BC604700BFB70E000056
:10B9400001B40248844601BC604700BFA94601001B
:10B9500001B40248844601BC604700BF594F010052
:10B9600001B40248844601BC604700BF595201003F
:10B9700001B40248844601BC604700BF8133FF1F09
:10B9800001B40248844601BC604700BF8B520100ED
:10B9900001B40248844601BC604700BFC94A0100A7
:10B9A00001B40248844601BC604700BF5125000035
:10B9B00001B40248844601BC604700BF4550000006
:10B9C00001B40248844601BC604700BFEDA50000F9
:10B9D00001B40248844601BC604700BFE92800006A
:10B9E00001B40248844601BC604700BF9DA9000025
:10B9F00001B40248844601BC604700BFC56D010028
:10BA000001B40248844601BC604700BF3D180000F5
:10BA100001B40248844601BC604700BFA54F010045
:10BA200001B40248844601BC604700BF7918000099
:10BA300001B40248844601BC604700BF456B010069
:10BA400001B40248844601BC604700BF156B010089
:10BA500001B40248844601BC604700BF090E0000E3
:10BA600001B40248844601BC604700BFADAE00008F
:10BA700001B40248844601BC604700BFD130FF1FBB
:10BA800001B40248844601BC604700BF8D2EFF1FF1
:10BA900001B40248844601BC604700BFF94C010074
:10BAA00001B40248844601BC604700BF8D1200000B
:10BAB00001B40248844601BC604700BFB54C010098
:10BAC00001B40248844601BC604700BFF30E000089
:10BAD00001B40248844601BC604700BF291C000035
:10BAE00001B40248844601BC604700BF3934FF1FDF
:10BAF00001B40248844601BC604700BF5D170000E6
:10BB000001B40248844601BC604700BF51470100B0
:10BB100001B40248844601BC604700BF0124000014
:10BB200001B40248844601BC604700BF4D2BFF1F93
:10BB300001B40248844601BC604700BF7536FF1F50
:10BB400001B40248844601BC604700BF11470100B0
:10BB500001B40248844601BC604700BFF933FF1FAF
:10BB600001B40248844601BC604700BF2146010081
:10BB700001B40248844601BC604700BF017F000059
:10BB800001B40248844601BC604700BF350E000086
:10BB900001B40248844601BC604700BF6DBC000090
:10BBA00001B40248844601BC604700BF3D4B010020
:10BBB00001B40248844601BC604700BF252600004E
:10BBC00001B40248844601BC604700BF1D4B010020
:10BBD00001B40248844601BC604700BF352DFF1FF9
:10BBE00001B40248844601BC604700BF0D2BFF1F13
:10BBF000000301030202030204020500060207001B
:10BC0000080009020A030B030C000D000E030F03CA
:10BC10001003110312031300140015031603000090
:10BC2000C13B0011F53B00110000000002000000C4
:10BC300036BC0011192A0F180A000000F159000043
:10BC4000FD240000414601004580001159A000116B
:10BC5000AD740011497E0011BD520011FDAD0011FF
:10BC6000254F0011B53D0011E53E00110000000018
:10BC7000161600000200000080BC0011F4FFF3FF64
:10BC8000D2FC000025400011000000000000000070
:10BC9000547579610042312E3400303031380067FC
:10BCA00069746875622E636F6D2F707676780054B4
:10BCB0004830350002000000C8BC0011292A282A9B
:10BCC000272A262A252A242A0A180000E20400002E
:10BCD0007102000078EC00007440000010270000A2
:10BCE00060F0000006640000204E0000000000002C
:10BCF000050000001F501D00023CB40000011800A8
:10BD000014000000A10200003031323334353637E0
:10BD1000383941424344454600000000C1560011F5
:10BD200015570011000000000200000034BD001192
:10BD30006F2A6E2A1A18EAD8BC80F0FC6000000056
:10BD40000000000000005F066B2F363D7D077F3F3F
:10BD5000777C596E7971AF066D4FC6CBEB0EEFCF86
:10BD6000EEC3A966E9E8FA60D6F46CBCBEE0FEFC5E
:10BD7000EE3E9A769E8E000001A0000000000000BA
:10BD80006410B71DC8206E3BAC30D9269041DC76DC
:10BD9000F4516B6B5861B24D3C7105502083B8ED86
:10BDA00044930FF0E8A3D6D68CB361CBB0C2649BAA
:10BDB000D4D2D38678E20AA01CF2BDBDFB349B5FCF
:10BDC000800000800010000000000000AF60001143
:10BDD00039770011D3600011417B001157610011C8
:10BDE000177B0011CD610011ED7A00111F62001167
:10BDF000B57C001187620011B57C0011B962001199
:10BE00006F7C0011CD610011A57A0011456200110F
:10BE10004D7C001100000000000000002B630011A9
:10BE20004D7C00118D63001151770011052A042A01
:10BE3000012A002A022903280128002801180018D5
:10BE4000000000000000000000000000000000876B
:10BE500001010201020101020102030304010301C5
:10BE6000010101010303020103000D000E00100097
:10BE7000110013001401070108010A010B011C0144
:10BE80001D02040205020702080219021A021C021E
:10BE90001D03010302031700020100050400080747
:10BEA000000B0A001716001D1C0102010105040108
:10BEB0000E0D011110011413011716011A190202B7
:10BEC00001020B0A020E0D021110021413021716C2
:10BED000030504030807030B0A030E0D0001020308
:10BEE00007090A0B0E0F101112141718191A1B1F2D
:10BEF0002021220045A7001101A800110000000028
:10BF0000020000003EBE0011000000002DB500112F
:0CBF100000000000020000003CBE001118
:020000041FFFDC
:10000000000000001D3D00113CBC001138BC001177
:10001000BC5BFF1F000000000000000000000000AB
:1000200000000000000000000000000000000000D0
:1000300000000000000000000000000000000000C0
:1000400000000000000000000000000000000000B0
:1000500000000000000000000000000000000000A0
:100060000000000000000000000000000000000090
:100070000000000000000000000000000000000080
:100080000000000000000000000000000000000070
:100090000000000000000000000000000000000060
:1000A0000000000000000000000000000000000050
:1000B0000000000000000000000000000000000040
:1000C0000000000000000000000000000000000030
:1000D0000000000000000000000000000000000020
:1000E0000000000000000000000000000000000010
:1000F0000000000000000000000000000000000000
:1001000000000000000000000000000000000000EF
:1001100000000000000000000000000000000000DF
:1001200000000000000000000000000000000000CF
:1001300000000000000000000000000000000000BF
:1001400000000000000000000000000000000000AF
:10015000000000000000000000000000000000009F
:10016000000000000000000000000000000000008F
:10017000000000000000000000000000000000007F
:10018000000000000000000000000000000000006F
:10019000812DFF1FE12BFF1FC16601000000000041
:1001A000000000000000000000000000000000004F
:1001B000000000000000000000000000000000003F
:1001C000000000000000000000000000000000002F
:1001D000000000000000000000000000000000001F
:1001E000000000000000000000000000000000000F
:1001F00000000000000000000000000000000000FF
:1002000000000000000000000000000000000000EE
:1002100000000000000000000000000000000000DE
:1002200000000000000000000000000000000000CE
:1002300000000000000000000000000000000000BE
:1002400000000000000000000000000000000000AE
:10025000000000000000000000000000000000009E
:10026000000000000000000000000000000000008E
:10027000000000000000000000000000000000007E
:10028000000000000000000000000000000000006E
:10029000000000000000000000000000000000005E
:1002A000000000000000000000000000000000004E
:1002B000000000000000000000000000000000003E
:1002C000000000000000000000000000000000002E
:1002D000000000000000000000000000000000001E
:1002E000000000000000000000000000000000000E
:1002F00000000000000000000000000000000000FE
:1003000000000000000000000000000000000000ED
:1003100000000000000000000000000000000000DD
:1003200000000000000000000000000000000000CD
:1003300000000000000000000000000000000000BD
:1003400000000000000000000000000000000000AD
:10035000000000000000000000000000000000009D
:10036000000000000000000000000000000000008D
:1003700079B500110000000000000000000000003E
:10038000000000000000000000000000000000006D
:10039000000000000000000000000000000000005D
:1003A000000000000000000000000000591AFF1FBC
:1003B000000000000000000000000000000000003D
:1003C000000000000000000000000000000000002D
:1003D000000000000000000000000000000000001D
:1003E000000000000000000000000000000000000D
:1003F00000000000000000000000000000000000FD
:08183800A069FF1F4118FF1F0A
:10184000024981F3088802F067F80000A069FF1FD1
:1018500010B501F021FF072804D0122808D0022873
:1018600008D010BD044A0420136B01331363F8E75A
:101870000220F6E71420F4E7885FFF1FF8B50700A1
:101880000C0026002500503630785135002804D150
:101890000300287058342370F8BD2978CA00481E08
:1018A0008141A3183800A25C5B68C9B2FFF7D0FF82
:1018B00000280DD12B78DA00A218013350602B706C
:1018C0003378044A013B3370136A01331362D8E75B
:1018D0000123DFE7885FFF1F5C234343074910B5FF
:1018E000C9180B0058331B78012B05D1FFF7C6FF31
:1018F000034A936A0133936210BDC046BC5FFF1F69
:10190000885FFF1F10B502F0C7F8064A01211300D7
:1019100010CB4942D967044B136002F075F82000E0
:1019200010BDC04600E100E01000100010B504003A
:1019300002F0B2F8024B1C6002F066F810BDC0461F
:1019400000E100E0431E5A425341A022F0B5D2010B
:101950005B421340154D164A40019B182A18127E0F
:101960008BB00191002A1BD01A000832D46F0022DC
:10197000E6B206AFE4B294420EDC2818C369002B2D
:1019800008D0019902AA117106AA049202AA16733C
:1019900003A898470BB0F0BD1978B9540132EAE7B3
:1019A0001A7D1A7806AB01261A70E6E74862FF1F17
:1019B00000400040F0B5254B04004001C25C85B0FA
:1019C000002A2BD01A18117E002927D0917E0029D9
:1019D00024D01179022921D11689D788D168F51B25
:1019E000ADB22A1C102D00D9102292B2BE4217D1DE
:1019F0001818012303710023C269C38003819A422E
:101A000006D06846032103730171029301A8904731
:101A10000820002C00D0192001F098F805B0F0BD86
:101A2000013C65426C41A0256442ED012C40084D0B
:101A30001B186419074D0633013A92B2AA42EDD041
:101A40001888461C1E80085C2070F5E74862FF1F5E
:101A500000400040FFFF00000F220E4B10B59868B9
:101A6000104002380A280BD801F0FAFD0D0A0B0AC3
:101A70000A110A0A0A0A060002210020FFF762FF83
:101A800010BD0121F9E70020FFF794FFF8E7DB6FB5
:101A9000F6E7C046004000400F220E4B10B5986894
:101AA000104002380A280BD801F0DAFD0E0A0B0AA2
:101AB0000A120A0A0A0A060002210120FFF742FF61
:101AC00010BD01210800F9E70120FFF773FFF7E7D8
:101AD000DB6FF5E700900040564B70B51B68012B9B
:101AE00003D1554A936D0133936501F00DFE534BBD
:101AF000534A1860534B544C1A600123534A1360E5
:101B0000534A13602378002B06D0062251495248CD
:101B100001F00AFF00232370504A514B10681B78D4
:101B2000C1B2002B0ED14F4CC0B223785BB2002B58
:101B30004FDB237824785BB264B21B0424021B19A8
:101B40001B1813600B1C50294ED95023464A474995
:101B50001078DBB2FF2202284BD10868444C454D77
:101B6000267890432A78964254D9227824782E7881
:101B7000023B5D10A31B6B435201D31A10335B1160
:101B80001843086001F0D8FE031F012B45D83A4BDB
:101B90001B78002B06D0394B1B78002B02D000207D
:101BA00001F022FEA122364B92009978354B4A4330
:101BB0001B689B18832292009B181B78033B012B08
:101BC00003D8AF20400001F0BFFE01222E4BDA8285
:101BD00070BD237824785BB264B2FF33FF341B04FA
:101BE00024021B190138ABE7CAB2022AAED2022383
:101BF000ACE70868254C264D267890432A78964213
:101C000008D9227824782D78023B5B10641B63434B
:101C10005201B2E72378DBB2B2E70228D5D11D4BDF
:101C20001B78013B022B03D91B4B1B78022BCCD119
:101C30006C20C8E79809FF1FFC0FFF1FC05EFF1F45
:101C4000FF3F000014100340C45EFF1F0C10034050
:101C500000100340D50BFF1F7211FF1FB40003409B
:101C60008C09FF1F680AFF1F490AFF1F94000340E9
:101C7000460AFF1F470AFF1FF908FF1F2209FF1F1F
:101C8000300DFF1F3409FF1FBC0BFF1F440AFF1F4D
:101C9000450AFF1F1C09FF1F2309FF1F10B501F094
:101CA0007BFE0022014B1A8010BDC046BC5EFF1FA8
:101CB00070B5244D2B68002B28D001F0D5FE2B6881
:101CC000D8402B680400002B27D001F055FE2B686C
:101CD000D8401D4B1D4A9978A1239B004B431268A5
:101CE000D118D25C91239B00002A20D0CA5801321F
:101CF000CA50174B17491B680868834214D3D23B5C
:101D0000181A012A1AD0144B186070BD01F0ACFEED
:101D1000124B196801F0F0FCD3E701F02DFE0F4BD8
:101D2000196801F0E9FCD4E70D495B18E8E7CA50EF
:101D30000C4B1B68DB68E418201AE4E7F530FF3031
:101D4000E1E7C0461C08FF1F300DFF1F3409FF1FCD
:101D50009C09FF1FC05EFF1FA009FF1F1808FF1F7F
:101D60002DFF3F00C85EFF1F70B504000D0028293D
:101D700016D10300A433C2881B889B1A0B4A9BB25E
:101D800093420DD906006A3605223100653001F014
:101D90008BFD002804D13100200001F0E5FD70BD6D
:101DA0002900200001F018FEF9E7C046FE7F000080
:101DB000F8B50500012001F0EFFC134CA36AA26AFC
:101DC0009342FBD1114E336001F0F6FC1049030041
:101DD00008601048426894460F4A17680022BC45C4
:101DE00001D24268BA1A0D4802603268AD18A422C6
:101DF000E562606A520302436262094A1278002A6D
:101E000001D00F3B0B60F8BD00F00040340AFF1F0B
:101E1000E408FF1F28100040180AFF1F1C0AFF1FBC
:101E20001C09FF1F70B580241025E405A3682B430F
:101E3000A36001F051FDA368AB43A36070BD000037
:101E4000F7B5160080221C001023D205019191687D
:101E500005000B43936000225A4BD7301A6001F003
:101E600023FE9D232A002F009B00EB58CA3201213C
:101E70000092FC37002B01D00021009A386801F055
:101E800003FD2900009BCB311A784F4BD3351A60E4
:101E90004B780A781B0213438A7812041A43CB78D2
:101EA0001B061343494A1BBA13604B790A791B027C
:101EB00013438A7912041A43CB7931001B0613436A
:101EC000434A1BBA13606B782A781B021343AA7823
:101ED00012041A43EB781B0613433E4A1BBA1360E5
:101EE000019A330213433C4A13603C4B22001B1BF4
:101EF0009C4603293DDCB3089A0013005142B21AF4
:101F0000032A46D1354AE018511A827840781204E3
:101F100000020243E05C043302430A600022FF2B0C
:101F20004BDDF0222E4B12011A600F222D4B1A604E
:101F30002D4A1368002BFCD00023224A2749136046
:101F4000091B321D0B191B68043A180A23706070B4
:101F5000180C1B0EA070E3700434002AF2DC8022FF
:101F600010213B68D20501333B6093688B4393603B
:101F7000F7BD6346D578981893782D061B042B433C
:101F8000157804392B43557804322D022B43036016
:101F9000AFE7022A0AD1114AE05C511AE2185278DE
:101FA000120202430A6004339BB2B7E7012AB5D19B
:101FB0000A4A521AE15C1160F5E7084959180A60AB
:101FC0000433ACE7000004403C0004403800044007
:101FD00034000440300004400C0004400001044080
:101FE000040004401000044014000440F7B515003C
:101FF00080221C001023D2050091916807000B433A
:1020000093600023654AD730136001F04DFD9D2396
:102010003E009B00F9583B00CA363200FC330029D1
:1020200000D07FE0586801F02FFC390032785C4B1B
:10203000CB311A604B780A781B0213438A78AC467E
:1020400012041A43CB78281D1B061343554A1BBAAA
:1020500013604B790A791B0213438A7912041A43DD
:10206000CB791B061343504A1BBA13604B7A0A7A8A
:102070001B0213438A7A12041A43CB7A21001B06EF
:1020800013434A4A1BBA1360009A2B021343484A6F
:1020900013602200474B1B1B0093009BCE785B18FC
:1020A00001938B7836061B0433430E780438334390
:1020B0004E78043136023343019E33600328ECDC52
:1020C0000321A808431C9B002940800003292BD131
:1020D0003849E5185E18A9786D78E35C09042D028B
:1020E000294319433160030008330021FF2B2DDD04
:1020F000314B324919600F21314B196001232749B7
:102100000B60304B19680029FCD006211B680B407E
:10211000042B20D080220020D20593680A318B4303
:102120009360FEBD01217DE7022908D121495D1898
:10213000E1184978E35C090219432960D3E70129D2
:10214000D3D11C495918E35C0B60CCE71948181827
:1021500001600433CAE7002310490B606346002B7B
:102160000CDC3B00FC335A68102101325A6080229B
:10217000D205936801208B439360D2E7009B9B18A4
:102180001B68190A13705170190C1B0ED3700423AD
:102190005B4291709C440432E0E7C046000004407A
:1021A0003C00044038000440340004403000044047
:1021B0000C0004400001044004000440080F00002B
:1021C000100004401400044010B5002901D001F0B3
:1021D0005BFC10BDF7B5604B01919978A1239B0082
:1021E0004B435E4A060014681022E418D6235B00B5
:1021F000E0583623FF33E35C00279343222B41D181
:10220000574B0F3A1A600760012501F035FB019B1F
:102210001880E8235B00E35C002B01D0B34258DD5B
:102220000023504FFB70AD33FF33E3581A68002A88
:1022300003D09B88DB439B071DD03823FF33E35C2F
:10224000002B18D09B235B00E35C002B13D1D13310
:10225000FF33E35CB3420EDAA4235B00E15AE018DB
:10226000090A023101F070FA23000122FE33013E17
:1022700001351A87FA70E8235B00E35C002B2AD053
:10228000A8B2FEBD03683D00002BBED0818804309B
:10229000090A023101F058FAD6235B00E3581F60A7
:1022A000B2E72300B133BA00FF3398580137818871
:1022B0000430090A023101F047FAE8235B00E35CCD
:1022C000BB42EEDCE822F61AED1800235200A354BC
:1022D000A6E70027F1E7200001F0F6FB00281FD059
:1022E000002E1DDD7319882647190193B6002000C2
:1022F00001F0FAF95A3080002018406801358188D1
:102300000430090A023101F01FFA200001F0ACFA92
:10231000A3590133A351BD4202D0019B9D42E6D196
:10232000114BE35C002BABD095239B00E35C002BAF
:10233000A6D00E4BE15A0029A2D00D4AA35C9942C7
:1023400002D90133A3549BE700231A212000A35490
:1023500001F03AFA94E7C046300DFF1F3409FF1F21
:1023600000140340E010FF1F5A0200007202000038
:102370005E0200000D4970B54A6E0D4CD2038B69A8
:10238000D20BA24206D80B4D0224AA4204D901F076
:1023900073FB70BD02246442E21815007E242540C0
:1023A0002242F4D0A3432B438B61F0E700F00040BE
:1023B0000A200000FC1C00000B001B3B70B5040051
:1023C0003020E02B0DD81300E025493BFF3B9BB2AA
:1023D000ED00AB4205D8034B200019825A8201F070
:1023E000FBF970BD8410FF1FD722044B92009B584D
:1023F00010B5002B00D0984710BDC0460000FF1F4D
:1024000010B501F0B7F8FFF7EFFF2749274BCA6D6A
:10241000274C1A4084235B001343CB65254B1B6874
:10242000186A01F0B9F9244B244A1A60244B254A52
:102430001A60A022244B52001A60244B187801F035
:1024400023F92000224901F0D7FA0023A3600233C8
:10245000A360204B2049236003232048A36001F0A0
:10246000CBFA10221E4BFF201A60802252031A6002
:10247000802292031A60802212041A6001F0B4F9DB
:10248000012001F009FAFA20400001F07DFA5820FD
:1024900001F05AFA134801F0C7FA012001F00CFAD2
:1024A000072001F019F910BD00F0004000FEFEFF0A
:1024B00014100040C85EFF1F000003400180063D6D
:1024C000BC00034034080000A40003404A0AFF1F78
:1024D00071020000C3090000FFFF3F002810004008
:1024E00000E100E0307500006B4E336888331B68F4
:1024F00083F3088801F030F9684A694913680020BD
:102500000B401360674B684A1B68934200D1ADE0F3
:1025100001F04AFA0221654A13688B431360FFF702
:102520006FFF634B634C1878C0B201F085F900234C
:10253000A3600233A360604B0120236001F02CF9FB
:102540000323A36001F068FA040001F0DDF8050040
:1025500001F062FA594B186001F0B6F9584B19684E
:10256000621A531EA14200D213008022D20393426A
:1025700001D39B029B0A3268D16AC90700D478E074
:1025800050491C0C09689BB24C4359432402090A68
:10259000641803274C49FC3293680A684B489B1A1D
:1025A0004B4A4C4E12684C499B184C4A34609A185E
:1025B0003B400193036892089C46019B0A60634478
:1025C0000360042B03D901323B400A6003600B68AF
:1025D0004349E418200001F08FF8424F40493B681E
:1025E000C3183B602000019301F076FA3E4C20684E
:1025F00008183B492060884205D9019B01333B60A4
:1026000001F06AFA216001F07FF9384B1B78002B4A
:102610000ED001F079F83168354B4A1B1B6812184F
:102620009A4233D2591A4919091A324801F0E4F989
:10263000314C237A002B0FD001F066F83168E36843
:102640004A1B1218934224D9591A4919091A2B48BE
:1026500001F0D2F900232372294B83F3088801F09B
:1026600093F8002001F0A0F901F0C6F801F09CF900
:1026700055E7DC0199000234641A5900641A0921F3
:102680004B438033CB40A408E41882E7FA21890049
:10269000CBE71C49DBE7C046C85EFF1F1CF00040CB
:1026A000FFFFC1FF0C0AFF1FB641210310000040CD
:1026B000490AFF1F14100040C3090000100AFF1F41
:1026C000340AFF1F380AFF1F200AFF1F280AFF1FB6
:1026D0001C0AFF1FB85EFF1F240AFF1FC409000069
:1026E000710200006008FF1F2C0AFF1F1C09FF1F5A
:1026F000E408FF1F00100040740BFF1F3C10004057
:1027000000000020DC050000A022054B92009B5831
:1027100010B5002B01D0984710BD01F09DF9FBE7E3
:102720000000FF1FA122054B92009B5810B5002B03
:1027300001D0984710BD01F08FF9FBE70000FF1FA3
:10274000A222054B92009B5810B5002B01D0984750
:1027500010BD01F081F9FBE70000FF1FA322054B2C
:1027600092009B5810B5002B01D0984710BD01F086
:1027700073F9FBE70000FF1FA422054B92009B5852
:1027800010B5002B01D0984710BD01F065F9FBE7AB
:102790000000FF1F70B500F0B7FF4F4B186001F04D
:1027A00043F80400C30702D400F0FEFF70BD00220E
:1027B0004A4B1A604A4B18780138042829D800F08F
:1027C0004FFF0320181C2400200001F00DF9012800
:1027D000ECD0444C2378042B6ED100F06DFF002820
:1027E000E4D001F081F8582001F0AEF80223237004
:1027F000DCE7200000F0C0FFE9E7200000F08CFFDC
:10280000E5E7200001F000F8E1E7200001F014F90D
:10281000DDE701F091F80500012808D1324B1B7863
:10282000053B012B03D82000FFF76EFFD1E72D4BAE
:102830001B78022B01D0052B20D1022D28D12B4B48
:102840009B7BAB431CD12000FFF76CFF264B187815
:102850000128BED16405BCD4244925224B7B034208
:1028600005D1233A13405A42534126331A000B7DB7
:102870009342AED9322001F09FF8AAE7022D07D18A
:10288000194B1B78052B11D12000FFF759FFDDE70D
:10289000012D0BD1012B03D12000FFF75FFF98E73B
:1028A000062B03D12000FFF767FF92E7200001F01D
:1028B000D3F8022D8DD1C9E7032B04D10C4B987CA2
:1028C00001F04AF872E7072B00D06FE7094B987BBD
:1028D00000F0FAFE6AE7C0469C09FF1F9809FF1F37
:1028E0009009FF1F2309FF1F1C09FF1FA60BFF1FD5
:1028F000BC0BFF1FD40BFF1F10B500F099FE10BDDD
:10290000F7B50B0CFF270122009300233C001E00AB
:102910001D009446019089B262469A40100008401A
:1029200018413618B6B2FF2F02D1012E00D19FB246
:10293000009802401A41AD18ADB2FF2C02D1012D12
:1029400000D19CB20133102BE6D10320012E07D118
:10295000012D04D1019B2401E4191C700138FEBD36
:10296000102EFCD10238102DF9D00230F7E700000C
:102970008023F7B59C46264B264F01932649274ACC
:10298000274D284C284B02281AD160463860086829
:10299000264E30408026360330430860019909787E
:1029A000002909D11660224A2A60224A2260E022C8
:1029B00019689143A03A1BE08021C9021160F2E737
:1029C00066463E600F68194E3E408027FF023E4338
:1029D0000E600199097800290DD1176001280ED1E8
:1029E000154A2A60154A2260E02219689143C03ACC
:1029F0000A431A60F7BD802189021160EEE7E021E9
:102A00000F4A02432A600F4A22601A688A43F0E79D
:102A10004B0AFF1FE0000340D80003409000034032
:102A2000000003405000034040000340FFFFE3FF6D
:102A30000280063D804508220180063D806608220E
:102A40000080069880550822F8B51E4B80261A682B
:102A5000002014003440324232D11A681A4F3243F7
:102A60001A6001223B68063093433B6000F094FEFD
:102A70000122164D2B681E432E603B680A26134325
:102A80003B608027BF00124B1B683B4211D1013EC7
:102A9000F6B2FF2E09D17E220E4B1C682B68E40B88
:102AA0001440934323432B6005E0082000F074FE9C
:102AB000E9E7002EEFD180222B68600893432B605A
:102AC000F8BDC046C4F000405CF0004018F0004083
:102AD00068F0004060F0004010B500F025FE0121D4
:102AE0005820034A00F098FEFFF7AEFF10BDC04625
:102AF000600AFF1F10B578220021034800F064FF30
:102B000000F032FE002010BDD061FF1F70B5040040
:102B100000F0C2FF00230C200B4A010059438D181E
:102B2000515C00290DD0A14208D1012300246B7013
:102B300000F0BAFD00F068FF200070BD01330A2BE1
:102B4000EBD11224F6E7C046D061FF1F70B5040038
:102B500000F0A2FF002319001D000D4A1078002884
:102B600006D0A0420CD1557001310C320A29F5D1A2
:102B7000002B0AD100F0F8FD00F046FF002070BDE8
:102B80005078461EB0411B18EEE700F08DFDF3E7CC
:102B9000D061FF1FF7B504000C20002384460E4DC2
:102BA000019267465F43E85D7E19A04212D000287B
:102BB0000BD10A4B9C4662461B7808331370019B6D
:102BC00070707C557160B360FEBD01330A2BE8D193
:102BD0000320F9E70720F7E7D061FF1FCC61FF1F53
:102BE0008020F8B5484BC0051B68C1248360474B63
:102BF000FF251A68012313434361454BA4001A685B
:102C0000444B40211A60444B1A68444B1A60444BB1
:102C10001A59AA431A51C52292009E58AE43314315
:102C2000802699509F583F49F6010F403E439E50E1
:102C30009E5880273602360A3043985080201A5911
:102C400000020A4002431A5104341A59364E3F0416
:102C5000324080263A431A511A5936061202120A95
:102C600032431A5108341A5980260A4002431A5135
:102C7000C32292009F58B446AF4337439F509F589A
:102C8000294E0F4007439F509F58374080263604F7
:102C9000374380269F509F5836063F023F0A3743EE
:102CA0009F50C0221F59AF433A431A511A5912027A
:102CB000120A1643C6221E5192009C58AC43654628
:102CC0002C439C509C5800250C4020439850C72012
:102CD00080001A58154C1140C02212020A431A50A3
:102CE000134B1B78DB08AB4201DC0020F8BD2378D6
:102CF000002B06D0A368002B00D0984701350C3478
:102D0000EEE71220F2E7C046E83DFF1FE43DFF1F5B
:102D1000B0F00040C861FF1FB4F00040C461FF1F65
:102D200000E100E0FF00FFFFFFFF00FFD061FF1F99
:102D3000CC61FF1F030010B51F2809D8072200200F
:102D40001340072404490A78A24313430B7010BDB3
:102D500000230620F5E7C046CC61FF1F054B06495E
:102D60001B780A6805485B0702401B0B13430020D1
:102D70000B607047CC61FF1F1CF00040FFFFC1FFDC
:102D800070B50C25FFF7EAFF0A4B1C780A4BE408E4
:102D90006543ED18002C01D1200070BD2B78002B6D
:102DA00006D06B68002B00D09847013C0C3DF1E742
:102DB0001220F2E7CC61FF1FC461FF1F1FB5002185
:102DC00002220B0001910091052000F03DFD02233D
:102DD0000B490A681A42FCD120230393039B5A1E15
:102DE0000392002BFAD1074A1368002BFCDA0B245C
:102DF0006C442000012100F07FFD207804B010BD5C
:102E000090C8004000C8004013B504000A4B01936D
:102E1000019B002B01D1112016BDFFF7CFFF23002E
:102E20000340044205D0052000F0B6FC019B013BA5
:102E3000EDE71800F0E7C046FFFFFF0707B500F019
:102E40002BFE80220821D205936A0191002B01D12B
:102E50000739916202210C4A11600199481E0190C4
:102E60000029FAD103311160053101910199481E01
:102E700001900029FAD11160002B02D18022D205E5
:102E8000936200F0C1FD07BD00C00040F0B52D4CBD
:102E900089B02378002B4FD1FEF734FD02232A4F4F
:102EA00003903A681A42FCD120230693069B5A1ECF
:102EB0000692002BFAD1254E3368002BFCDA012054
:102EC000FFF7A2FF011E02D0112009B0F0BD0300E0
:102ED00003220190009005AD9F2000F0B5FC032176
:102EE000280000F009FD02233A681A42FCD1202391
:102EF0000793079B5A1E0792002BFAD13368002BC9
:102F0000FCDA0120FFF780FF0028DDD10398FEF7EF
:102F10000DFDAA786B7811041B020B4329780B4333
:102F200063601300113B0A49052B07D80123934026
:102F3000A3600B60012323700020C6E780231B03DE
:102F4000F6E7C046D03DFF1F90C8004000C80040D3
:102F50009808FF1F1E4B30B55A6818781D4B85B076
:102F6000D31859424B4101210093002300F074FC17
:102F7000194B1A4A02259A6300221A6510325A65C3
:102F80008022C4219D65164B1648D202DA6789005B
:102F90004258154B80241A4080231B04134343508E
:102FA000642341200393E40500F006FA402000F07A
:102FB00003FA6562039D6B1E0393002DFAD1032370
:102FC0006362FFF73BFFA562FFF760FF05B030BD0E
:102FD000DC3DFF1F95FFFEF700C80040050001FF24
:102FE00004E100E000E100E0FFFF00FFF0B585B084
:102FF0000700FEF787FC022305002D4C22681A42C9
:10300000FCD120230093009B5A1E0092002BFAD182
:10301000284E3368002BFCDA0120FFF7F5FE00286C
:1030200003D01124200005B0F0BD234B2360022300
:1030300022681A42FCD120230193019B5A1E01925F
:10304000002BFAD13368002BFCDA0120FFF7DCFEFD
:103050000028E6D1194B1F60022322681A42FCD1D6
:1030600020230293029B5A1E0292002BFAD133684E
:10307000002BFCDA0120FFF7C7FE0028D1D1104B4E
:103080002360022322681A42FCD120230393039B6E
:103090005A1E0392002BFAD13368002BFCDA012070
:1030A000FFF7B2FE041EBCD12800FEF73FFCB9E7D3
:1030B00090C8004000C8004001000006A8C80040B9
:1030C0000180000110B50020FFF790FF10BD000047
:1030D00010B5064B18705960FFF73CFF0021132014
:1030E000034AFFF757FD002010BDC046DC3DFF1F1F
:1030F000552FFF1FF0B5040085B003920291FEF733
:1031000001FC882263035B0B52051A438023DB0515
:103110009D6A8023274F0092BA68002601901B0306
:103120009A420CD9F82326001B041E401C4206D0EC
:103130008022214B52025E6219680A431A60002DF8
:103140000BD100F0A9FC02221C4B1A608023DB0586
:103150005A62013A9A6200F057FC0023039A9342A4
:1031600020D1002D0AD100F097FC144B03221D60E2
:103170008023DB055A629D6200F046FC8023BA681A
:103180001B039A4208D9002E06D000220A4B0C4994
:103190005A621A680A401A600198FEF7C7FB0020BD
:1031A00005B0F0BD009A0299D2181278CA540133C2
:1031B000D4E7C046D03DFF1F00C8004000C000401B
:1031C000FFFFFEFFF0B587B0029103920400FEF707
:1031D00099FB019000F060FC802302250122234E20
:1031E000DB0535605D629A6200F00EFC204F3B68A3
:1031F0002B42FCD120230493049B5A1E0492002BE3
:10320000FAD11C4D2B68002BFCDA0120FFF7FCFDE6
:10321000002802D0112007B0F0BD2000039A0299C7
:1032200000F04AFC022304003A681A42FCD1202331
:103230000593059B5A1E0592002BFAD12B68002B93
:10324000FCDA0120FFF7E0FD051EE3D100F024FCCD
:1032500080230322DB0535605A629D6200F0D4FBB7
:103260000198FEF763FBE0B2D5E7C04600C000401E
:1032700090C8004000C80040F0B5802489B0060026
:10328000FEF740FBE405A36A02250393029000F0D9
:1032900003FC0123304F3D606562A36200F0B4FB84
:1032A0002E4C23682B42FCD120230593059B5A1EEC
:1032B0000592002BFAD12A4D2B68002BFCDA012055
:1032C000FFF7A2FD002803D01124200009B0F0BDB3
:1032D000244B2360022322681A42FCD12023069348
:1032E000069B5A1E0692002BFAD12B68002BFCDAA3
:1032F0000120FFF789FD021EE6D11B4B03211E6052
:10330000030001900090202000F09EFA0223226822
:103310001A42FCD120230793079B5A1E0792002BC9
:10332000FAD12B68002BFCDA0320FFF76DFD041E99
:10333000CAD100F0B1FB80230322DB053C605A6256
:103340009C6200F061FB039B002B01D1FFF776FD2F
:103350000298FEF7EBFAB8E700C0004090C80040C2
:1033600000C800400100000694C8004007B50002F4
:1033700001910422000A01A9FFF724FF0EBD0000FD
:1033800073B5050005240B4AA3005B429B1819681E
:103390006B46DE1D3000FFF7B3FA022804D1337804
:1033A0002B55013CEFD276BD052CFCD00128FAD17B
:1033B0000230F8E7140900111F2807D801238022E2
:1033C0008340D20591680B43936070473F2808D82B
:1033D0000123802220388340D20551690B43536179
:1033E000F3E75F28F1D80123802240388340D205DB
:1033F000116A0B431362E8E71F2807D801228021D6
:103400008240C9058B6893438B6070473F2808D87A
:103410000122802120388240C9054B6993434B61CA
:10342000F3E75F28F1D80122802140388240C905A6
:103430000B6A93430B62E8E71F2810D88023020031
:10344000DB05153A1968012A06D820229143196034
:1034500019680A431A60704701228240F6E73F2844
:1034600011D880230200DB05353AD968032A06D833
:1034700010229143D960D9680A43DA60EBE7012250
:1034800020388240F5E75F28E5D842238022181AC9
:10349000413B8340D205516A99435162516A0B43C3
:1034A0005362D8E710B50400012813D1A0221849AF
:1034B00092050B685B015B0913430B60154B164AC1
:1034C00019681140154A0A431A60402219680A43D4
:1034D0001A6010BD0028FCD101000A2000F02CF970
:1034E00021000B2000F028F9C0220A4B9200196835
:1034F0000A4340211A601A688A431A60B0220449BC
:1035000012060B685B015B0913430B60E1E7C046E1
:1035100014F000401CF000407F00FEFF80FD010021
:1035200072B6074A1368013313600422054B1A6010
:103530000023054A13608022D2055360FEE7C0468F
:103540007808FF1FC0F00040C4F0004005490B6838
:10355000002B05D1044A0A6004490A60044A13603A
:103560007047C046140AFF1F841E0000380AFF1F60
:10357000C4F000400023034A1360034A1360034A67
:103580001360704754F0004040F1004044F10040A7
:10359000002310B5184C8AB0009301932378012BB7
:1035A00027D06946012000F04FFA002817D1009B70
:1035B00012490293019B06AA0393114B02A81B68B0
:1035C0000493104B1B68059300F086F910220E49F6
:1035D00006A800F069F9002804D1FF232370002019
:1035E0000AB010BD0123094A074902A8237000F060
:1035F00073F90120F4E7C046CC5EFF1F10290011CB
:10360000082900110C29001120290011D05EFF1F8C
:1036100013B501246946012000F016FA034B00940B
:103620000193FFF7B5FF200016BDC046BB0B00009D
:1036300010B5FFF79FFFFFF7EBFF002802D0024B0A
:10364000984710BDFEE7C046E1A2000002B47146F3
:1036500049084900095649008E4402BC7047C046DB
:1036600002B4714649084900095C49008E4402BC15
:103670007047C04603B47146490840004900095AE2
:1036800049008E4403BC704701B40248844601BC23
:10369000604700BFEDA5000001B40248844601BCAC
:1036A000604700BFE927000001B40248844601BC1E
:1036B000604700BF21A9000001B40248844601BC54
:1036C000604700BF01D7000001B40248844601BC36
:1036D000604700BFC1F7000001B40248844601BC46
:1036E000604700BFF90D010001B40248844601BCE7
:1036F000604700BFD9B0000001B40248844601BC55
:10370000604700BF090E000001B40248844601BCB6
:10371000604700BFC95C010001B40248844601BC97
:10372000604700BF0534010001B40248844601BC73
:10373000604700BFED68010001B40248844601BC47
:10374000604700BF29A2001101B40248844601BCB1
:10375000604700BFC115010001B40248844601BCA6
:10376000604700BFC9A9000001B40248844601BCFB
:10377000604700BFADAE000001B40248844601BC02
:10378000604700BF0934010001B40248844601BC0F
:10379000604700BF7997000001B40248844601BC2D
:1037A000604700BF0189000001B40248844601BCA3
:1037B000604700BFDD0A010001B40248844601BC35
:1037C000604700BFBD5C010001B40248844601BCF3
:1037D000604700BF53B9000001B40248844601BCF1
:1037E000604700BF116E000001B40248844601BC6E
:1037F000604700BFED6B010001B40248844601BC84
:10380000604700BF8552010001B40248844601BCF4
:10381000604700BFF535010001B40248844601BC91
:10382000604700BF0167010001B40248844601BC43
:10383000604700BFBD0B010001B40248844601BCD3
:10384000604700BF8914010001B40248844601BCEE
:10385000604700BF496D010001B40248844601BCC5
:10386000604700BFC56D010001B40248844601BC39
:10387000604700BF5976010001B40248844601BC8C
:10388000604700BFCD0C010001B40248844601BC72
:10389000604700BF2144000001B40248844601BCD7
:1038A000604700BF6911010001B40248844601BCB1
:1038B000604700BFCD4C010001B40248844601BC02
:1038C000604700BFE512010001B40248844601BC14
:1038D000604700BFC166010001B40248844601BCD4
:1038E000604700BFDD3F000001B40248844601BCD0
:1038F000604700BF6DF6000001B40248844601BC79
:10390000604700BF3D71010001B40248844601BC1C
:10391000604700BFD544010001B40248844601BCA1
:10392000604700BF81B5001101B40248844601BC64
:10393000604700BFE94C010001B40248844601BC65
:10394000604700BFDD0C010001B40248844601BCA1
:10395000604700BF7912010001B40248844601BCEF
:10396000604700BF4DF9000001B40248844601BC25
:10397000604700BF85C1000001B40248844601BC15
:10398000604700BF6D0B010001B40248844601BCD2
:10399000604700BF8512010001B40248844601BCA3
:1039A000604700BF8D82000001B40248844601BC1C
:1039B000604700BF016C010001B40248844601BCAD
:1039C000604700BF6137010001B40248844601BC72
:1039D000604700BFB70E000001B40248844601BC36
:1039E000604700BF51B8000001B40248844601BCE2
:1039F000604700BF0134010001B40248844601BCA5
:103A0000604700BF2D6C010001B40248844601BC30
:103A1000604700BF9DA9000001B40248844601BC74
:103A2000604700BF156B010001B40248844601BC29
:103A3000604700BF8D11010001B40248844601BCFB
:103A4000604700BFF935010001B40248844601BC5B
:103A5000604700BFE1AC000001B40248844601BCED
:103A6000604700BFE917010001B40248844601BC69
:103A7000604700BFE90B010001B40248844601BC65
:103A8000604700BFD1AE000001B40248844601BCCB
:103A9000604700BFE9D4000001B40248844601BC7D
:103AA000604700BF75A9000001B40248844601BC0C
:103AB000604700BF8944000001B40248844601BC4D
:103AC000604700BF9573010001B40248844601BC01
:103AD000604700BF71B0000001B40248844601BCD9
:083AE000604700BF090E000061
:103AE800020000003ABE0011010000002CBC0011C9
:103AF8000200000036BE001101000000283BFF1F35
:103B08000200000034BC0011010000003C5CFF1FF3
:103B18000200000034BE001103000000B05BFF1F6C
:103B280012000000020000003ABE0011010000006F
:103B380074BC00110200000036BE00110100000034
:103B480071BC0011020000007EBC001103000000DF
:103B5800EB5BFF1F0200000034BE001103000000F1
:103B6800005CFF1F0200000036BE001101000000CB
:103B780070BC0011020000007CBC001103000000B2
:103B8800C15BFF1F0200000034BE001103000000EB
:103B9800E25BFF1F020000003ABE001101000000B6
:103BA800B4BC00110200000036BE00110100000084
:103BB800713CFF1F02000000C6BC0011010000009C
:103BC800AFBC00110200000036BE00110100000069
:103BD800703CFF1F02000000C4BC0011010000007F
:103BE800085CFF1F0200000036BE00110100000043
:103BF8006F3CFF1F02000000C2BC00110100000062
:103C08009FBC00110200000036BE00110100000038
:103C18006E3CFF1F02000000C0BC00110100000044
:103C28009ABC00110200000036BE0011010000001D
:103C38006D3CFF1F02000000BEBC00110100000027
:103C480095BC00110200000036BE00110100000002
:103C58006C3CFF1F02000000BCBC0011010000000A
:103C680090BC0011020202020202000000000000E3
:103C780014130000694B00112F4B001108BD0011EF
:103C880090011D0018001800FFFF0701020304053A
:103C9800060201060000000000000000000000000D
:103CA800000000000000000000000000000000000C
:103CB80003000000020000003ABE001101000000ED
:103CC80028BD00110200000036BE001101000000EE
:103CD8002C3DFF1F0200000032BD00110100000052
:103CE800365CFF1F0200000034BE00110300000014
:103CF800A05EFF1F0200000036BE00110100000098
:103D08002C3DFF1F0200000030BD00110100000023
:103D1800385CFF1F0200000034BE001103000000E1
:103D2800985EFF1F12006C6C00000000000000008D
:103D38000000000008070000000100000000011159
:103D4800FFFF000050485936000000000000000046
:103D58000B000500F0000000B4000028002800282F
:103D68003075A000A000A000A00000080008E00135
:103D7800F00010001000100010001000100050009B
:103D88005000500010001000D00700000000000094
:103D98000F0001000500307507001000010081FFC9
:103DA80000000000FF0000001174001119720011DA
:103DB800A96F0011FFFF0100FF0000002D9E0011F8
:103DC800A99B0011C19A001100000000000000002A
:103DD80000000800040000003B0001085902E0014F
:103DE80088212800020000003ABE001101000000EE
:103DF80000BF00110200000036BE001101000000E3
:103E0800693EFF1F0200000032BE001101000000E1
:103E18008862FF1F0200000036BE0011010000008A
:103E2800683EFF1F0200000030BE001101000000C4
:103E3800663EFF1F0200000036BE001101000000B0
:103E4800643EFF1F020000002EBE001101000000AA
:103E58005C3EFF1F180018001D00900102000003BF
:103E680002020000020000003ABE0011010000003A
:103E780014BF00110200000036BE0011010000004E
:103E8800AC3EFF1F020000002CBE00110000000025
:103E9800000000000200000034BE00110300000012
:063EA800A862FF1F20FFCD
:040000051FFF184180
:00000001FF
